:100000000C9463000C948B000C948B000C948B006C
:100010000C948B000C9452200C948B000C948B004D
:100020000C948B000C948B000C948B000C948B0024
:100030000C948B000C948B000C948B000C948B0014
:100040000C94E91E0C948B000C94B71E0C94911E1A
:100050000C948B000C948B000C948B000C948B00F4
:100060000C94331F0C948B00000000002400270028
:100070002A0000000000250028002B0000000000DE
:1000800023002600290004040404040404040202DA
:100090000202020203030303030301020408102007
:1000A0004080010204081020010204081020000012
:1000B0000008000201000003040700000000000027
:1000C0000000CD20C63111241FBECFEFD8E0DEBF27
:1000D000CDBF27E0A8EDB4E001C01D92A733B20761
:1000E000E1F714E0A0E0B1E0E2EEF1E702C0059034
:1000F0000D92A83DB107D9F710E0C2E6D0E004C0E8
:100100002197FE010E94E336C136D107C9F70E944C
:10011000AB210C94E4380C940000982F2091FA0540
:1001200081E0213208F043C08091D6058111FCCFD7
:100130008091F90532E03093D6059093D5059FEF75
:100140009093D4051092D3052093D205A9EDB5E084
:10015000E2EBF5E090E0291331C01092B1059091E7
:10016000B105880F892B8093B1058091B00581304E
:1001700049F51092B0058091B1058093BB00809144
:10018000BC0083FDF8CF85EC8093BC008091D60540
:100190008230E1F38091D4058F3FB1F08091D40596
:1001A0008032A1F08091D405803391F084E01092E8
:1001B000D8051092FA051092D70508953D91319314
:1001C0009F5FC9CF85EEE0CF80E0F1CF82E0EFCF37
:1001D00083E0EDCF80918E0590918F05891B990B5F
:1001E0000895089508952F923F924F925F926F92D3
:1001F0007F928F929F92AF92BF92CF92DF92EF92B7
:10020000FF920F931F93CF93DF93CDB7DEB76C9719
:100210000FB6F894DEBF0FBECDBF522E3D874E877E
:10022000252E462E372E782E692EA982BF86C88AA3
:10023000D98AEA8AFB8A0C8B1D8B988E8F8A2115AE
:1002400000EA30070CEA400709EB500703E06007BB
:1002500071058105910509F098F52F3F10EE3107E2
:1002600015EF410715E051076105710581059105FD
:1002700009F008F40BC12F3F354D41415E47634003
:1002800071058105910509F008F40BC129813F85AD
:10029000488959896A897B898C899D89A0E099243C
:1002A00093940E94C336C9F4F1E0FE8B04E0802EE3
:1002B000912CA12CB12C89869A86AB86BC8616C15E
:1002C000512CB0EABD87ECEAEE8789EB282E93E04B
:1002D000492E312C712C612CD9CFA52CBD84CE8414
:1002E000D22CE42CF32C072D162D29813F8548892B
:1002F00059896A897B898C899D890E940E36298754
:100300003A874B875C8729853A854B855C85B6E0C3
:10031000AB2EB12C263031054105510568F0898599
:100320009A85AB85BC8589309740A105B105E0F081
:10033000F8E0AF2EA7E0BA2EC12CD12CE12CF12C85
:1003400000E010E029813F85488959896A897B89C5
:100350008C899D890E940E36522E3D874E87252E10
:10036000462E372E782E692EA52CBD84CE84D22C15
:10037000E42CF32C072D162D29813F8548895989B6
:100380006A897B898C899D890E940C36AA24AA944B
:10039000BB24BA94EFE0CE2ED12CE12CF12C00E05E
:1003A00010E00E944935A52CBD84CE84D22CE42CCB
:1003B000F32C072D162D0E940E36A32FF42FE52FB8
:1003C000422F5A2F6F2F7E2FCC24CA94DC2C8FE023
:1003D000E82EF12C411551056105710521F4C12C60
:1003E000D12C7601C394AA24A3949A1409F4E5C0ED
:1003F00001E00E8BCB01BA0137E0660F771F881F33
:10040000991F3A95D1F7A70196010E940835298FC7
:100410003A8F4B8F5C8F89849A84AB84BC8447E08D
:10042000880C991CAA1CBB1C4A95D1F79501840124
:1004300012502109310948015901298D3A8D4B8DFE
:100440005C8D280D391D4A1D5B1DAF89B88D2D931C
:100450003D934D935C931397FD016483758386836D
:1004600097831896CD92DD92ED92FC921B978E8821
:10047000882009F481C059829D849F86AE84A88A11
:10048000298A4A8A3B8A7C8A6D8A76C0512C01EE81
:100490000D8715EF1E8725E0222E412C312C712C63
:1004A000612C29813F85488959896A897B898C8992
:1004B0009D89A0E0912C0E94C33609F00ECFA52C97
:1004C000BD84CE84D22CE42CF32C072D162D20E0F5
:1004D00034E04BE654EF64E170E080E090E00E948D
:1004E0000E3629873A874B875C871E8A89849A84CF
:1004F000AB84BC84A501940160E070E0CB01A52C25
:10050000BD84CE84D22CE42CF32C072D162D298308
:100510003A834B835C836D837E838F83988760E00F
:1005200070E080E090E00E94493529833F87488B46
:10053000598B6A8B7B8B8C8B9D8B0E89C12CD12C1C
:100540007601C39440E050E0BA01013009F052CF87
:10055000AF89B88D1D921D921D921C921397FD01BB
:10056000148215821682178281E090E0A0E0B0E04C
:1005700080879187A287B38729813F8548895989D8
:100580006A897B898C899D896C960FB6F894DEBF49
:100590000FBECDBFDF91CF911F910F91FF90EF90D4
:1005A000DF90CF90BF90AF909F908F907F906F9093
:1005B0005F904F903F902F900895AF89B88D1D9216
:1005C0001D921D921C921397FD01148215821682B2
:1005D000178281E090E0A0E0B0E080879187A28759
:1005E000B3875982FD85FF878E84888A49CFDF9241
:1005F000EF92FF920F931F93CF93DF93FC01E08064
:10060000F18002811381D481C581B681D7809701A1
:10061000A8016D2F7C2F8B2F9D2D35534C405109F8
:1006200061097109810991092F3F34434C405105FB
:10063000610571058105910509F0D0F49701A801C4
:100640006D2F7C2F8B2F9D2D07E00E947B36208302
:10065000318342835383648375838683978387E0E2
:10066000DF91CF911F910F91FF90EF90DF90089550
:100670009701A8016D2F7C2F8B2F9D2D3A56484155
:10068000510961097109810991092F3F3946484192
:100690005105610571058105910509F098F49701EF
:1006A000A8016D2F7C2F8B2F9D2D06E00E947B369D
:1006B0002083318342835383648375838683978346
:1006C00086E0CECF9701A8016D2F7C2F8B2F9D2D1B
:1006D000345D4043510961097109810991092F3F36
:1006E000334D40435105610571058105910509F0C0
:1006F00098F49701A8016D2F7C2F8B2F9D2D05E07D
:100700000E947B36208331834283538364837583C5
:100710008683978385E0A4CF9701A8016D2F7C2F56
:100720008B2F9D2D385A4146510961097109810964
:1007300091092F3F374A41465105610571058105F1
:10074000910509F098F49701A8016D2F7C2F8B2F4C
:100750009D2D04E00E947B362083318342835383A6
:10076000648375838683978384E07ACF9701A80199
:100770006D2F7C2F8B2F9D2D3055434C51096109D6
:100780007109810991092F3F3F44434C510561058F
:1007900071058105910509F098F49701A8016D2F65
:1007A0007C2F8B2F9D2D03E00E947B36208331838D
:1007B00042835383648375838683978383E050CF1A
:1007C0009701A8016D2F7C2F8B2F9D2D305A464805
:1007D000514061097109810991092F3F3F494648FC
:1007E0005140610571058105910509F098F4970163
:1007F000A8016D2F7C2F8B2F9D2D02E00E947B3650
:1008000020833183428353836483758386839783F4
:1008100082E026CF9701A8016D2F7C2F8B2F9D2D75
:1008200030544D40534061097109810991092F3FAE
:100830003F434D405340610571058105910509F025
:1008400098F49701A8016D2F7C2F8B2F9D2D01E02F
:100850000E947B3620833183428353836483758374
:100860008683978381E0FCCE80E0FACE0895DB0199
:1008700014964D915C9115976D917C91DC01ED91F1
:10088000FC910280F381E02D0994AF92BF92CF9248
:10089000DF92EF92FF920F931F93CF93DF936C0140
:1008A0007B018B01040F151FEB015E01AE18BF0821
:1008B000C017D10759F06991D601ED91FC910190D3
:1008C000F081E02DC6010995892B79F7C501DF91EB
:1008D000CF911F910F91FF90EF90DF90CF90BF903D
:1008E000AF900895FC01538D448D252F30E0842F67
:1008F00090E0821B930B541710F0CF960895019748
:100900000895FC01918D828D981761F0A28DAE0F34
:10091000BF2FB11D5D968C91928D9F5F9F73928FBB
:1009200090E008958FEF9FEF0895FC01918D828DE7
:10093000981731F0828DE80FF11D858D90E00895B4
:100940008FEF9FEF0895FC01918D228D892F90E00C
:10095000805C9F4F821B91098F73992708958BEFBD
:1009600095E00E94A30421E0892B09F420E0822F66
:10097000089580E090E0892B29F00E94AF04811156
:100980000C9400000895FC01A48DA80FB92FB11D8F
:10099000A35ABF4F2C91848D90E001968F739927B5
:1009A000848FA689B7892C93A089B1898C91837093
:1009B00080648C93938D848D981306C00288F3898C
:1009C000E02D80818F7D80830895EF92FF920F93B9
:1009D0001F93CF93DF93EC0181E0888F9B8D8C8DEB
:1009E00098131AC0E889F989808185FF15C09FB7DF
:1009F000F894EE89FF896083E889F98980818370A2
:100A0000806480839FBF81E090E0DF91CF911F9150
:100A10000F91FF90EF900895F62E0B8D10E00F5F71
:100A20001F4F0F731127E02E8C8D8E110CC00FB647
:100A300007FCFACFE889F989808185FFF5CFCE01DF
:100A40000E94C304F1CFEB8DEC0FFD2FF11DE35A93
:100A5000FF4FF0829FB7F8940B8FEA89FB89808162
:100A60008062CFCFCF93DF93EC01888D8823B9F0DC
:100A7000AA89BB89E889F9898C9185FD03C08081A9
:100A800086FD0DC00FB607FCF7CF8C9185FFF2CF26
:100A9000808185FFEDCFCE010E94C304E9CFDF91B5
:100AA000CF910895833081F028F4813099F082301D
:100AB000A9F008958730A9F08830C9F08430B1F4E6
:100AC000809180008F7D03C0809180008F7780931C
:100AD0008000089584B58F7784BD089584B58F7D97
:100AE000FBCF8091B0008F778093B0000895809104
:100AF000B0008F7DF9CFCF93DF93282F30E0F9013D
:100B0000E255FF4F8491F901E656FF4FD491F90168
:100B1000EA57FF4FC491CC23A1F081110E945205E6
:100B2000EC2FF0E0EE0FFF1FE458FF4FA591B491BA
:100B3000EC91ED2381E090E009F480E0DF91CF912A
:100B4000089580E090E0FACF1F93CF93DF93282F92
:100B500030E0F901E255FF4F8491F901E656FF4F6D
:100B6000D491F901EA57FF4FC491CC23A9F0162F75
:100B700081110E945205EC2FF0E0EE0FFF1FEE589E
:100B8000FF4FA591B4918FB7F894EC91111108C063
:100B9000D095DE23DC938FBFDF91CF911F91089515
:100BA000DE2BF8CF10928F0510928E051092D8058B
:100BB0001092FA051092D60581E08093D505109227
:100BC000B00561E082E10E94A40561E083E10E943A
:100BD000A405E9EBF0E080818E7F808380818D7FAA
:100BE000808388E48093B80085E48093BC0081EF23
:100BF00090E090938D0580938C0582EF90E0909328
:100C00008B0580938A050895CF93DF9390E0FC01D4
:100C1000E656FF4F24918A579F4FFC018491882309
:100C2000C9F090E0880F991FFC01E859FF4FA5918A
:100C3000B491FC01EE58FF4FC591D49161110DC0E4
:100C40009FB7F8948C91209582238C9388812823D8
:100C500028839FBFDF91CF910895623051F49FB7F1
:100C6000F8943C91822F809583238C93E8812E2BDE
:100C7000EFCF8FB7F894EC912E2B2C938FBFEACF48
:100C80008E50806480937C0080917A008064809391
:100C90007A0080917A0086FDFCCF80917800909157
:100CA000790008953FB7F894809124059091250527
:100CB000A0912605B091270526B5A89B05C02F3F1A
:100CC00019F00196A11DB11D3FBFBA2FA92F982F72
:100CD0008827BC01CD01620F711D811D911D42E06D
:100CE000660F771F881F991F4A95D1F708958F9235
:100CF0009F92AF92BF92CF92DF92EF92FF924B0101
:100D00005C010E9452066B017C010E9452066C1924
:100D10007D098E099F09683E734081059105A8F3FE
:100D200021E0821A9108A108B10888EEC80E83E07C
:100D3000D81EE11CF11C81149104A104B10429F70F
:100D4000FF90EF90DF90CF90BF90AF909F908F90EB
:100D500008952FB7F8946091200570912105809136
:100D60002205909123052FBF089585ED8093BC0047
:100D70008091BC0084FDFCCF1092D605089520918F
:100D8000FC04260F3327331F21323105ECF4209168
:100D9000D605FC0190E080E0243069F082E00895FF
:100DA000A091FC042191AC0144525B4FA40FB52FDC
:100DB000B11D2C930196861798F38091FC04680F5F
:100DC0006093FC0480E0089581E008950895E09127
:100DD0008F0580918E05E81730F4F0E0E057FA4F68
:100DE000808190E008958FEF9FEF089590918F0597
:100DF00080918E052FEF3FEF981748F4E92FF0E030
:100E0000E057FA4F208130E09F5F90938F05C90132
:100E10000895CF92DF92EF92FF920F931F93CF939B
:100E2000DF937C01CB018A012091D705222389F031
:100E3000EB016B01C40ED51ECC15DD0569F069917F
:100E4000D701ED91FC910190F081E02DC70109954A
:100E5000F3CF642F0E94BF06C801DF91CF911F918D
:100E60000F91FF90EF90DF90CF900895CF93DF9395
:100E70001F92CDB7DEB769832091D7052223F9F001
:100E80002091FA05203258F021E030E0FC01338354
:100E9000228390E080E00F90DF91CF9108958091C0
:100EA000D805E82FF0E0E752FA4F998190838F5FE1
:100EB0008093D8058093FA0581E090E0ECCF61E063
:100EC000CE0101960E94BF06F7CFCF93C62F91E0C7
:100ED0009093D70590E69093F9051092D80510925B
:100EE000FA05682F88E996E00E9436076C2F88E99A
:100EF00096E00E94360781E0CF910C948D000F930D
:100F00001F93CF93DF938B0191E09093D70590E6E9
:100F10009093F9051092D8051092FA05682F88E988
:100F200096E00E943607E801085F1F4F699188E943
:100F300096E00E943607C017D107C1F781E0DF9124
:100F4000CF911F910F910C948D0090E080E0089557
:100F50008FE00E9440069093600580935F05BC017E
:100F6000990F880B990B0E94483220E030E040EA4C
:100F700050E40E94A73220E030E040E85AE30E94AB
:100F8000A7326093D8047093D9048093DA049093C5
:100F9000DB040895CF93DF9391E09093D70590E61B
:100FA0009093F9051092D8051092FA05682F88E9F8
:100FB00096E00E94360781E00E948D008091D60560
:100FC0008111FCCF81E08093D6051092D5059FEF6B
:100FD0009093D4051092D3051092D2058093B10559
:100FE0008091B105806C8093B1058091B00581300E
:100FF00061F51092B0058091B1058093BB0080919E
:10100000BC0083FDF8CF85EC8093BC008091D605B1
:101010008130E1F38091D305811119C08091D3050E
:10102000E2EBF5E0A0E9B5E0C0E0C81312C0109211
:101030008F05C0938E0580918F05C81771F088E9E0
:1010400096E00E94F606D82FF6CF85EEDDCF81E040
:10105000E7CF91919D93CF5FE8CF8D2FDF91CF9117
:101060000895CF93C0E1C80F8C2F0E94CA07682F44
:1010700063608C2FCF910C946507CF93DF93D82FAB
:10108000C62F83E00E94CA0761E070E001C0660FCE
:10109000DA95EAF7C13039F46095682383E0DF918F
:1010A000CF910C946507682BF9CF0F931F93CF93C3
:1010B0008B01C0E1C80F8C2F0E94CA07682F012B3B
:1010C00039F46F7D8C2FCF911F910F910C94650790
:1010D0006062F8CFCF93DF93EC0160E08E810E94D5
:1010E000A40561E08E810E94A40560E08E810E94CB
:1010F000A4058BE891E00197F1F7DF91CF91089576
:10110000CF92DF92EF92FF920F931F93CF93DF93D3
:101110006C017C0187E0E80EF11CD0E0C0E0062FF6
:1011200010E0B8010C2E02C0759567950A94E2F79D
:101130006170F70181917F010E94A4052196C4305E
:10114000D10579F7C601DF91CF911F910F91FF90E3
:10115000EF90DF90CF900C946A08CF92DF92EF92DD
:10116000FF920F931F93CF93DF93EC01F62E642F22
:101170008C810E94A4058D818F3F19F060E00E9450
:10118000A4050F2D10E08F8584FF25C06E0187E038
:10119000C80ED11CF12CE12CB8010E2C02C07595A3
:1011A00067950A94E2F76170F60181916F010E94E0
:1011B000A405FFEFEF1AFF0A88E0E816F10461F7D3
:1011C000CE01DF91CF911F910F91FF90EF90DF90B3
:1011D000CF900C946A08B80184E0759567958A955C
:1011E000E1F7CE010E9480086F2DCE01DF91CF91F3
:1011F0001F910F91FF90EF90DF90CF900C9480089B
:1012000040E0682F8BE197E00C94AD08CF93DF931B
:10121000823029F490912A07986090932A0780934E
:101220002E0710922F0780E48093300780E180938F
:10123000310780E58093320761E080911F070E94AB
:101240000406809120078F3F19F061E00E94040698
:1012500061E0809121070E940406CBE1D7E09E0166
:101260002B51374080912A0784FD0BC084E090E029
:1012700021962817390744F461E08E810E94040604
:10128000EECF88E090E0F4CF8BE39DE00197F1F79B
:1012900060E080911F070E94A40560E08091210713
:1012A0000E94A405809120078F3F19F060E00E9402
:1012B000A40580912A0784FD39C063E08BE197E0A3
:1012C0000E948008CBE4D6E4CE010197F1F763E0F9
:1012D0008BE197E00E9480082197F1F763E08BE1B2
:1012E00097E00E94800883E592E00197F1F762E0C1
:1012F0008BE197E00E94800880912A0780620E941B
:10130000000984E080932B078CE00E94000981E0B3
:101310000E9400098BE39FE10197F1F782E080933F
:101320002C0786E0DF91CF910C94000980620E9427
:1013300000098BE496E40197F1F780912A07806217
:101340000E94000983E592E00197F1F780912A0756
:1013500080620E940009D0CF90912E07691710F08B
:101360006FEF690FE62FF0E0E55EF84F9489890F83
:1013700080680C94000941E00E94AD0881E090E093
:1013800008950F931F93CF93DF938B0128E0829FE3
:10139000C001112480640E940009E801085F1F4F0A
:1013A00069918BE197E00E94BB09C017D107C1F793
:1013B000DF91CF911F910F91089541E0682F8BE14C
:1013C00097E00E94AD0881E090E00895FC01019053
:1013D0000020E9F73197AF01481B590BBC018BE1A5
:1013E00097E00C9445048F929F92AF92BF920F9317
:1013F0001F93CF93DF93CDB7DEB7A1970FB6F894C5
:10140000DEBF0FBECDBF19A2423008F44AE08E0104
:101410000F5D1F4F842E912CB12CA12CA50194019E
:101420000E940835E62FB901CA01EA30F4F4E05D04
:10143000D801EE938D01232B242B252B79F790E0F7
:1014400080E0109719F0CD010E94E609A1960FB631
:10145000F894DEBF0FBECDBFDF91CF911F910F91EA
:10146000BF90AF909F908F900895E95CE1CFCF92AD
:10147000DF92EF92FF92CF93DF9397FF19C06B013A
:101480007C018DE20E94DD09EC0166277727CB0104
:101490006C197D098E099F094AE00E94F3098C0F9F
:1014A0009D1FDF91CF91FF90EF90DF90CF90089537
:1014B0004AE0DF91CF91FF90EF90DF90CF900C94B6
:1014C000F3090C94E609CF92DF92EF92FF92C0905D
:1014D0004105D0904205E0904305F09044058AE034
:1014E000C816D104E104F1041CF480E20E94DD0975
:1014F00080E20E94DD09C701B6010E94370A8EE230
:101500000E94DD096091450570914605809147056F
:101510009091480520E432E44FE050E00E942A35E3
:1015200028EE33E040E050E00E942A3569017A015C
:10153000C0924105D0924205E0924305F0924405E5
:1015400084E6C816D104E104F10464F480E30E9447
:10155000DD098AE0C816D104E104F1041CF480E33B
:101560000E94DD09C701B6010E94370A8EE20E947F
:10157000DD09609145057091460580914705909180
:10158000480528EE33E040E050E00E942A356B0128
:101590007C01C0924105D0924205E0924305F09251
:1015A000440584E6C816D104E104F10464F480E340
:1015B0000E94DD098AE0C816D104E104F1041CF49C
:1015C00080E30E94DD09C701B6010E94370A83E665
:1015D00094E0FF90EF90DF90CF900C94610A80919F
:1015E0003D0590913E0561E0019709F451C080E00E
:1015F0000E94AC098091840190918501A09186019F
:10160000B091870184369105A105B10591F190F45F
:101610008A309105A105B10531F182339105A1050B
:10162000B10521F10197A105B105C1F586E192E06F
:101630000C94610A883E23E09207A105B105F9F0F8
:1016400030F4843F9140A105B105B1F00895803197
:1016500027E29207A105B105A9F0803A9648A1407A
:10166000B10599F008958BE192E0E2CF80E292E03B
:10167000DFCF85E292E0DCCF8AE292E0D9CF8FE241
:1016800092E0D6CF84E392E0D3CF89E392E0D0CF4B
:1016900080E00E94AC098EE392E0CACF089561E039
:1016A00084E00E94AC096091BB017091BC01809103
:1016B000BD019091BE0160934505709346058093EE
:1016C00047059093480520E432E44FE050E00E9443
:1016D0002A352093410530934205409343055093AA
:1016E00044050E94630A89EE92E00C94610A61E06D
:1016F00084E00E94AC096091B6017091B7018091BD
:10170000B8019091B90160934505709346058093A7
:1017100047059093480520E432E44FE050E00E94F2
:101720002A35209341053093420540934305509359
:1017300044050E94630A89EE92E00C94610A4F927C
:101740005F926F927F928F929F92AF92BF92CF9251
:10175000DF92EF92FF920F931F93CF936B017C0167
:10176000742EAC019B010E94DF34882399F083E43E
:1017700092E0CF911F910F91FF90EF90DF90CF906B
:10178000BF90AF909F908F907F906F905F904F90A1
:101790000C94E60946015701E894B7F82FEF3FEFA4
:1017A0004FE75FE7C501B4010E94DF3481110DC02E
:1017B0002FEF3FEF4FE75FE7C501B4010E944132D1
:1017C00018161CF487E492E0D4CF2FEF3FEF4FE7D9
:1017D0005FE4C701B6010E94DA3418161CF48BE4EA
:1017E00092E0C7CF2FEF3FEF4FE75FECC701B601A5
:1017F0000E94413287FDF3CF20E030E0A901C7010C
:10180000B6010E94413210E000E087FF08C08DE27F
:101810000E94DD098C01F7FAF094F7F8F094C0E02B
:1018200060E070E080E09FE37C1641F020E030E073
:1018300040E251E40E943934CF5FF6CFA701960110
:101840000E94CD332B013C010E94AB344B015C0163
:101850004AE00E94F3097C01E00EF11ECC23B1F1B5
:10186000C501B4010E9446329B01AC01C301B20123
:101870000E94CC334B015C018EE20E94DD09E80E30
:10188000F91EC15018F120E030E040E251E4C501FA
:10189000B4010E94A7322B013C010E94AB344B01E2
:1018A000B12CA12C4AE0C501B4010E94F309E80E55
:1018B000F91EC501B4010E9446329B01AC01C3016F
:1018C000B2010E94CC334B015C01DBCFC701CF9149
:1018D0001F910F91FF90EF90DF90CF90BF90AF904E
:1018E0009F908F907F906F905F904F9008952F9270
:1018F0003F924F925F926F927F928F929F92AF92A0
:10190000BF92CF92DF92EF92FF920F931F93CF93EC
:10191000DF93CDB7DEB72D970FB6F894DEBF0FBEBD
:10192000CDBF3C01C982DA82EB82FC820D831E832B
:101930002F83388749875A876B877C878AA18D8751
:101940003C2C2D2C9E2C502E412EB22EC984DA8494
:10195000EB84FC8484E190E00E94E9368C01FC0178
:10196000D082C182862D880F880F880F845D0E94E7
:10197000CA07F92DF3709F2E8C7F982AF801928266
:10198000238234824CE0F694E794D794C7944A9526
:10199000D1F7FC2DF07FCF2E8B2D8F70C82AF80148
:1019A000C58246825782B80182E3F1E06F16710466
:1019B00031F082E06816710409F447C08AE20E949F
:1019C0007F0730E1F32EF60C8F2D0E94CA0791E0BD
:1019D000682FA9123CC060648F2D0E946507E1E06A
:1019E0006E167104B1F1F2E06F167104B9F1A092B4
:1019F0000E072CE2F22E8F2D0E94CA0783789D8558
:101A000091118C60E0E18E9EB0011124682B8F2D26
:101A10000E946507C8012D960FB6F894DEBF0FBE71
:101A2000CDBFDF91CF911F910F91FF90EF90DF908D
:101A3000CF90BF90AF909F908F907F906F905F906E
:101A40004F903F902F900C9485378AE3B8CF6F7BEF
:101A5000C3CFA0920F0794E3F92ECDCFA092100729
:101A60008CE3F82EC8CF2F923F924F925F926F92E5
:101A70007F928F929F92AF92BF92CF92DF92EF921E
:101A8000FF920F931F93CF93DF93CDB7DEB76A9783
:101A90000FB6F894DEBF0FBECDBF2F8B3987488FAE
:101AA000598F6A877A8F1C011E8B0D8B60911707E7
:101AB000709118078091190790911A0724E630E079
:101AC00040E050E00E94B035522E632E742E852ED9
:101AD000962E788B8F87492E80911107909112074F
:101AE000A0911307B09114076C017D01FF0CCC0885
:101AF000DC2C76019C01AD016C2D7C2D8C2D9C2D58
:101B00000FE10E947B36A12CEAECBE2EFAE9CF2E23
:101B1000ABE3DA2EE12CF12C00E010E00E94DD3581
:101B2000A52CB62CC72CD82CE92CF8880F85142DA1
:101B30000E9449350FE10E94963629833A834B83F0
:101B40005C836D837E838F83988789819A81AB8143
:101B5000BC81BB0F880B982FDC018B879C87AD87DE
:101B6000BE87252D362D472D582D692D7F2D8F852C
:101B7000942DA980BA80CB80DC80EB84FE2C0E2DC6
:101B80001E2D0E94B13629833B874F87588B698B66
:101B90007A8B8B8B9C8B8F889A8C282D3985488DDE
:101BA000598D6A85792DC101211534404B46544F1A
:101BB000644171058105910569F060F0812CB4E004
:101BC000B987EBE6E88FF4EFF98F84E18A87912CEF
:101BD000212C312C282D3985488D598D6A85792DF8
:101BE000C101211538454744584F6D4071058105A5
:101BF000910560F4812CB8E5B987E7E4E88FF8EF48
:101C0000F98F8DE08A87912C212C312CA980BB84FF
:101C1000CF84D888E988FA880B891C89282D3985D2
:101C2000488D598D6A85792DC1010E940E36290192
:101C30003A011FE0A12E9FE049165104610471048E
:101C400040F0ABE54A16510461047104D0F0BAE5E6
:101C5000AB2EB12CC12CD12CE12CF12C00E010E0EA
:101C600029813B854F85588969897A898B899C8927
:101C70000E944935822E3987488F598F6A87972E5F
:101C80001C01A980BB84CF84D888E988FA880B8995
:101C90001C89282D3985488D598D6A85792DC1017A
:101CA0000E940C36AA24AA94BB24BA94AFE0CA2E90
:101CB000D12CE12CF12C00E010E00E944935A980E4
:101CC000BB84CF84D888E988FA880B891C890E9454
:101CD0000E36C901DA01812C912C540183940097AE
:101CE000A105B10531F088248A94982CEFE0AE2E3E
:101CF000B12CBC01CD0127E0660F771F881F991F0B
:101D00002A95D1F7A50194010E940835362E272E79
:101D1000182F67E0440C551C661C771C6A95D1F798
:101D2000B2E05B1A61087108420E531E641E751EF4
:101D300084E190E00E94E9369A838983FC019082D5
:101D40008182862D83708283538244827CE0B694A4
:101D5000A794979487947A95D1F7F82DF07F8F2EDA
:101D6000812AA981BA8115968C92159716962C9284
:101D7000169717963C921797ED89FE89BD018AE167
:101D8000EF2B19F069817A8182E20E947F078981B5
:101D90009A816A960FB6F894DEBF0FBECDBFDF9171
:101DA000CF911F910F91FF90EF90DF90CF90BF9058
:101DB000AF909F908F907F906F905F904F903F90EB
:101DC0002F900C9485372F923F924F925F926F9293
:101DD0007F928F929F92AF92BF92CF92DF92EF92BB
:101DE000FF920F931F93CF93DF93CDB7DEB7AA97E0
:101DF0000FB6F894DEBF0FBECDBF622E298F732EB3
:101E00003A8F4B8F5C8F6D8F7E8F8F8F98A319A722
:101E100008A793012F3F34434C40510561057105DC
:101E20008105910509F050F4198E85E38A8F8CE0C5
:101E30008B8F1C8E1D8E1E8E1F8E18A2298D3A8DA3
:101E40004B8D5C8D6D8D7E8D8F8D98A12115304AC7
:101E50004C4A594B634071058105910569F060F06A
:101E6000198E80EA8A8F8CEA8B8F89EB8C8F83E0C6
:101E70008D8F1E8E1F8E18A2CE0149960E94F702EA
:101E80008FA3798CBA8DAB8DFC8DED8D6E8C5F8CB4
:101E900048A0272D3B2F4A2F5F2F6E2F762D852DA3
:101EA000942D2F3F05ED300701E140070EE7500765
:101EB00003E0600771058105910511F008F09EC0EF
:101EC000CE010D964C01A12CE4E0BE2EFBE6CF2EF8
:101ED000A4EFDA2EB4E1EB2EF12C00E010E0852D1A
:101EE000942D0E94F300798D6A8D5B8D4C8D3D8D14
:101EF0002E8D9F8D88A1E8A5F9A5E130F10509F4A3
:101F000045C0329709F45EC07093F6066093F706F9
:101F10005093F8064093F9063093FA062093FB0697
:101F20009093FC068093FD0680E019A2412CF4E01A
:101F3000FAA30BE60BA314EF1CA394E19DA3512C71
:101F4000612C712C8F938FA0A82ECD84DE84EF841A
:101F5000F88809891A892B893C894D895E896F899E
:101F6000788D88A599A50E94770C0F9099A1913042
:101F700009F0FBC08101242D3AA14BA15CA16DA108
:101F8000752DC3010E94330D19A2EFC07093FE0698
:101F90006093FF06509300074093010730930207B8
:101FA00020930307909304078093050780E019A20C
:101FB000412CE4E0EAA3FBE6FBA304EF0CA314E14D
:101FC0001DA3BDCF709306076093070750930807C2
:101FD0004093090730930A0720930B0790930C074F
:101FE00080930D0780E019A2412C94E09AA3EBE6C0
:101FF000EBA3F4EFFCA304E10DA3A1CFCE010D965A
:102000004C01A12CB12CC12CD12CE12CF12C00E0E5
:1020100010E0852D942D0E94F300298C3A8CBB8D05
:10202000AC8DFD8DEE8D08A519A50130110509F4C3
:102030004EC00230110509F4A5C100E010E0910185
:102040004B2F5A2F6F2F7E2F8F8D98A10E94F30058
:10205000422E3AA34BA35CA36DA3572E3C0170E024
:1020600060E090E080E00E9455084092E6069AA168
:102070009093E706EBA1E093E806FCA1F093E90654
:102080000DA10093EA065092EB066092EC06709266
:10209000ED06898D8093F6068A8D8093F7068B8DE9
:1020A0008093F8068C8D8093F9068D8D8093FA06C7
:1020B0008E8D8093FB068F8D8093FC0688A1809384
:1020C000FD0681E011E019A3312C212C3BCF0F8DAF
:1020D00009A318A11EA310911607123009F019C107
:1020E00091014B2F5A2F6F2F7E2F802F9EA130589A
:1020F0004A41564061097109810991092F37304ED3
:1021000042475849624071058105910509F008F47C
:1021100046C020910607309107074091080750916B
:10212000090760910A0770910B0780910C07909145
:102130000D075101CB2EDA2EEF2EFE2E09A11EA186
:102140000E94BA3661F11092FE061092FF061092BC
:1021500000071092010710920207109203071092D5
:1021600004071092050711E019A389A1AA960FB6DA
:10217000F894DEBF0FBECDBFDF91CF911F910F91BD
:10218000FF90EF90DF90CF90BF90AF909F908F9097
:102190007F906F905F904F903F902F900895409068
:1021A000EE068091EF068AA39091F0069BA3009122
:1021B000F1060CA31091F2061DA35090F306609057
:1021C000F4067090F506CE010D964C01A42CBAA031
:1021D000CBA0D02EE12EF52C830191014B2F5A2F4D
:1021E0006F2F7E2F89A19EA10E94F30061E070E015
:1021F00081E090E00E94550819A2298D3A8D4B8DFF
:102200005C8D6D8D7E8D8F8D98A130584A415640E2
:1022100061097109810991092F37304E42475849A8
:10222000624071058105910509F008F4A7C081E0BD
:102230008093160720910607309107074091080701
:102240005091090760910A0770910B0780910C0764
:1022500090910D07A0E00E94C336F1F186E097E06F
:102260000E94F7028FA3A090EE06B090EF06C090F8
:10227000F006D090F106E090F206F090F30600919F
:10228000F4061091F506209106073091070740915A
:1022900008075091090760910A0770910B07CE015A
:1022A00001964C0180910C0790910D070E94F3005C
:1022B0001F928FA0A12CC980DA80EB80FC800D8159
:1022C0001E812F81388549855A856B857C8582E002
:1022D00090E00E94770C0F90898D8093FE068A8D86
:1022E0008093FF068B8D809300078C8D8093010770
:1022F0008D8D809302078E8D809303078F8D809341
:10230000040788A18093050781E022242394312CBF
:1023100019CE2093EE063093EF064093F0065093CB
:10232000F1066093F2067093F3068093F40690939F
:10233000F5068E01035F1F4F4801A12CB12CC12C63
:10234000D12CE12CF12C00E010E091014B2F5A2F01
:102350006F2F7E2F89A19EA10E94F300422E3AA3E7
:102360004BA35CA36DA3572E3C0161E070E081E0BC
:1023700090E00E94550811E019A33FCF88E08093B8
:102380001607AACF0091160709A31F8D1EA308A147
:102390000AA719A1113009F0F9C091014B2F5A2F4A
:1023A0006F2F7E2F8EA1902F30584A4156406109E1
:1023B0007109810991092F37304E424758496240CF
:1023C00071058105910561F158F120910607309161
:1023D0000707409108075091090760910A0770911B
:1023E0000B0780910C0790910D075101CB2EDA2E2F
:1023F000EF2EFE2E0EA11AA50E94BA3689F0109279
:10240000060710920707109208071092090710920A
:102410000A0710920B0710920C0710920D07A5CE19
:102420004090EE061091EF061AA38091F0068BA360
:102430009091F1069CA30091F2060DA35090F30633
:102440006090F4067090F506CE010D964C01A42C18
:10245000B12ECBA0DCA0E02EF52C830191014B2FF7
:102460005A2F6F2F7E2F8EA19AA50E94F30061E054
:1024700070E082E090E00E94550819A2298D3A8D03
:102480004B8D5C8D6D8D7E8D8F8D98A130584A411E
:10249000564061097109810991092F37304E424731
:1024A0005849624071058105910509F008F4A3C0FF
:1024B00082E0809316072091FE063091FF0640913E
:1024C0000007509101076091020770910307809106
:1024D000040790910507A0E00E94C336F1F18EEF4A
:1024E00096E00E94F7028FA3A090EE06B090EF0650
:1024F000C090F006D090F106E090F206F090F3065E
:102500000091F4061091F5062091FE063091FF0629
:1025100040910007509101076091020770910307F5
:10252000CE0101964C0180910407909105070E940D
:10253000F3001F928FA0A12CC980DA80EB80FC8071
:102540000D811E812F81388549855A856B857C8553
:1025500081E090E00E94770C0F90898D80930607B0
:102560008A8D809307078B8D809308078C8D8093CD
:1025700009078D8D80930A078E8D80930B078F8DB1
:1025800080930C0788A180930D07BECE2093EE06A2
:102590003093EF064093F0065093F1066093F206F5
:1025A0007093F3068093F4069093F5068E01035F13
:1025B0001F4F4801A12CB12CC12CD12CE12CF12CA6
:1025C00000E010E091014B2F5A2F6F2F7E2F8EA12C
:1025D0009AA50E94F300422E3AA34BA35CA36DA3DD
:1025E000572E3C0161E070E082E090E00E945508C7
:1025F00011E019A343CF88E080931607AECFCF93A5
:10260000DF93EC0188819981009711F00E94853752
:10261000198218821D821C821B821A82DF91CF913F
:102620000895FC01808191810C9485370F931F934D
:10263000CF93DF938C01EB010E9465338883C8013F
:1026400001960E9465338983CE01DF91CF911F915E
:102650000F910895CF92DF92EF92FF920F931F9305
:10266000CF93DF93EB017B0124E0E20EF11C8B01A1
:102670006C01C61AD70AC601800F911F0E946533EC
:10268000F80181938F01EE15FF05A9F7CE01DF91C7
:10269000CF911F910F91FF90EF90DF90CF90089511
:1026A000CF93DF93C0913705D091380568E271E090
:1026B0008AEA90E0209739F0C130D105E1F564E273
:1026C00071E08FEA90E00E942A13FC0180819181E1
:1026D000A281B3818093C0019093C101A093C201F4
:1026E000B093C301109251051092520510925305F8
:1026F0001092540564E171E083EC90E0C530D1059F
:10270000C1F50E942A13FC0180819181A281B381CD
:102710008093C0019093C101A093C201B093C30103
:1027200010925105109252051092530510925405C3
:10273000DF91CF910895C230D10519F560E271E0C3
:1027400084EB90E00E942A13FC0180819181A28198
:10275000B3818093C0019093C101A093C201B09353
:10276000C301109251051092520510925305109218
:10277000540560E171E088EC90E0C630D10509F2C3
:102780001EC0C330D10561F56CE171E089EB90E0CA
:102790000E942A13FC0180819181A281B3818093E0
:1027A000C0019093C101A093C201B093C3011092E4
:1027B00051051092520510925305109254056CE089
:1027C00071E08DEC90E0C730D10509F49ACF68E054
:1027D00071E082ED90E0C830D10509F492CF1FC0BE
:1027E000C430D10509F086CF68E171E08EEB90E04E
:1027F0000E942A13FC0180819181A281B381809380
:10280000C0019093C101A093C201B093C301109283
:1028100051051092520510925305109254052997B4
:1028200009F086CF64E071E087ED90E06ACFCF9346
:10283000DF93EB010E9465338883CE01DF91CF9156
:1028400008950F931F93CF93DF93EC0188819981B3
:10285000009759F02A813B812617370730F081E035
:10286000DF91CF911F910F9108958B016F5F7F4F83
:102870000E940E38009759F0998388831B830A833E
:102880002C813D81232B59F7FC011082E8CF80E099
:10289000E7CFEF92FF920F931F93CF93DF936115D2
:1028A000710541F480E0DF91CF911F910F91FF906E
:1028B000EF90089541155105B1F07B01EC010C81B9
:1028C0001D81040F151FB8010E942114882351F3A4
:1028D000288139818C819D81B701820F931F0E94CD
:1028E000DD381D830C8381E0DECFFC0101900020E8
:1028F000E9F73197AF01481B590BBC018CEB96E00F
:102900000C944914EF92FF920F931F93CF93DF9390
:10291000EC017B018A01BA010E94211481110BC0D4
:10292000CE010E94FF12CE01DF91CF911F910F9136
:10293000FF90EF9008951D830C83B70188819981E2
:102940000E94DD38F0CFFB0101900020E9F73197BC
:10295000AF01461B570B0C948214FC0111821082AC
:102960001382128215821482FB0101900020E9F784
:102970003197AF01461B570B0C948214FF920F93B3
:102980001F93CF93DF93EC01F62E08811981C801C4
:102990000E946533F81621F06F2DC8010E946D3337
:1029A000CE01DF91CF911F910F91FF900895EF928B
:1029B000FF920F931F93CF93DF9300D0CDB7DEB775
:1029C00000EC11E0805C91407C01C701800F911FF9
:1029D0009A838983F80161918F01CE0101960E944B
:1029E000BE14F1E0043C1F0781F780EC91E00F90EA
:1029F0000F90DF91CF911F910F91FF90EF9008956D
:102A00004091C0015091C1016091C2017091C30118
:102A10008091730590917405A0917505B09176052C
:102A2000481759076A077B0709F4BFC08091C001A6
:102A30009091C101A091C201B091C3018031974230
:102A4000A105B105B8F08091C0019091C101A0919C
:102A5000C201B091C301803C964CAD42B10550F427
:102A600015B810923805109237058AEA90E00E9456
:102A7000D7148BC08091C0019091C101A091C20177
:102A8000B091C301803C964CAD42B10570F080918D
:102A9000C0019091C101A091C201B091C3018034E5
:102AA0009B44AC44B10508F481C08091C001909171
:102AB000C101A091C201B091C30180349B44AC44D8
:102AC000B10508F07EC08091C0019091C101A09134
:102AD000C201B091C30181159241AA47B10508F026
:102AE00089C08091C0019091C101A091C201B091B3
:102AF000C30181159B41A74BB10508F094C080919B
:102B0000C0019091C101A091C201B091C301811592
:102B10009442A44FB10508F09FC08091C0019091EC
:102B2000C101A091C201B091C301803C9A4EA14263
:102B3000B14008F0AAC08091C0019091C101A0915C
:102B4000C201B091C3018038914BAF44B14008F04D
:102B5000B5C08091C0019091C101A091C201B09116
:102B6000C301803C9C4FAB49B14008F0C0C080918C
:102B7000C0019091C101A091C201B091C301811522
:102B80009A45A246B24008F0CBC08091C001909116
:102B9000C101A091C201B091C301809373059093CC
:102BA0007405A0937505B0937605089584E085B902
:102BB00081E090E090933805809337058FEA90E0AC
:102BC00056CF8091C0019091C101A091C201B091F6
:102BD000C30181159241AA47B10508F074CF88E07E
:102BE00085B982E090E0909338058093370584EBB7
:102BF00090E03DCF8091C0019091C101A091C201B0
:102C0000B091C30181159B41A74BB10508F069CF75
:102C10008CE085B983E090E0909338058093370588
:102C200089EB90E024CF8091C0019091C101A091E7
:102C3000C201B091C30181159442A44FB10508F0BF
:102C40005ECF80E185B984E090E090933805809371
:102C500037058EEB90E00BCF8091C0019091C101C0
:102C6000A091C201B091C301803C9A4EA142B140F3
:102C700008F053CF84E185B985E090E09093380562
:102C80008093370583EC90E0F2CE8091C001909163
:102C9000C101A091C201B091C3018038914BAF44F2
:102CA000B14008F048CF88E185B986E090E0909384
:102CB00038058093370588EC90E0D9CE8091C0012B
:102CC0009091C101A091C201B091C301803C9C4F81
:102CD000AB49B14008F03DCF8CE185B987E090E089
:102CE00090933805809337058DEC90E0C0CE8091AD
:102CF000C0019091C101A091C201B091C3018115A1
:102D00009A45A246B24008F032CF80E285B988E009
:102D100090E0909338058093370582ED90E0A7CE40
:102D20008091C0019091C101A091C201B091C301F5
:102D30008130924CAB4EBB4008F027CF84E285B97E
:102D400089E090E0909338058093370587ED90E017
:102D50008ECEEF92FF920F931F93CF93DF9300D00D
:102D6000CDB7DEB78C017B019A838983FB0160813B
:102D7000CE0101960E94BE140F5F1F4F1A83098374
:102D8000F7016181CE0101960E94BE14C7010F9028
:102D90000F90DF91CF911F910F91FF90EF900895C9
:102DA0000F931F93CF93DF938091880590918905AE
:102DB000019701F560E080E00E94AC098FE492E0A9
:102DC0000E94610A0E94EF0A61E084E00E94AC095F
:102DD00082E694E00E94610A6091340170913501AD
:102DE00080913601909137010E94370A81E994E081
:102DF0000E94610A8091880590918905029761F48B
:102E00000E94770B60E080E00E94AC0981E692E0CE
:102E10000E94610A0E94EF0A8091880590918905BD
:102E20000397F9F46BEB71E082E090E00E942A13C3
:102E3000FC0180819181A281B3818093BB01909339
:102E4000BC01A093BD01B093BE010E944F0B60E096
:102E500080E00E94AC0982E792E00E94610A0E9431
:102E6000EF0A80918805909189050497E1F560E06B
:102E700080E00E94AC0983E892E00E94610A8091A0
:102E8000BF01811117C064E972E080EB96E00E94F7
:102E9000A31461E080E00E94AC0960EB76E08BE176
:102EA00097E00E94370480E20E94DD0988E992E001
:102EB0000E94610A8091BF018130A9F468EA72E042
:102EC00080EB96E00E94A3140E944F0B61E080E02B
:102ED0000E94AC0960EB76E08BE197E00E9437043A
:102EE00080E20E94DD09809188059091890505970F
:102EF00009F049C060E080E00E94AC098CEA92E0F1
:102F00000E94610A8091BA01811117C064E972E0E0
:102F10008AEA96E00E94A31461E080E00E94AC0976
:102F20006AEA76E08BE197E00E94370480E20E9433
:102F3000DD0988E992E00E94610A8091BA0181303E
:102F4000A9F468EA72E08AEA96E00E94A3140E945B
:102F5000770B61E080E00E94AC096AEA76E08BE1E1
:102F600097E00E94370480E20E94DD0961E080E082
:102F70000E94AC096AEA76E08BE197E00E94370490
:102F800080E20E94DD09809188059091890506976D
:102F900001F560E080E00E94AC098DEB92E00E94B8
:102FA000610A0E94EF0A61E084E00E94AC0982E6B7
:102FB00094E00E94610A60916F05709170058091A4
:102FC0007105909172050E94370A8EEC92E00E9482
:102FD000610A8091880590918905079709F560E05D
:102FE00080E00E94AC0987ED92E00E94610A61E0F6
:102FF00080E00E94AC098DE694E00E94610A609135
:1030000030017091310180913201909133010E9421
:10301000370A88EE92E00E94610A80E20E94DD0990
:1030200080918805909189050897D1F460E080E04F
:103030000E94AC098CEE92E00E94610A61E080E09F
:103040000E94AC0981E994E00E94610A64EA76E09A
:103050008BE197E00E94370489E794E00E94610ABF
:103060008091880590918905099709F01AC280918D
:10307000A8069091A906892B09F413C2C091A40651
:10308000D091A50664E972E0CE010E94D438892B64
:1030900021F4109289051092880568EA72E0CE0149
:1030A0000E94D438892B09F0F2C10E94A906009130
:1030B0006105109162052091630530916405601BE4
:1030C000710B820B930B653F71408105910508F4EC
:1030D000DEC161E080E00E94AC098DEF92E00E94C9
:1030E000610A6091D8047091D9048091DA049091BA
:1030F000DB0442E00E949F0B8EE693E00E94610A8F
:10310000809131058130C1F40E94A80760E080E021
:103110000E94AC0989E093E00E94610A80915F05FA
:103120009091600590932F0180932E016EE271E0E3
:1031300084E690E00E94A916809131058230D1F595
:103140000E94A80760E080E00E94AC098BE193E058
:103150000E94610A80915F059091600590938D01B6
:1031600080938C0120912E0130912F01821B930BB3
:1031700063E070E00E94F434260F371F30932D0176
:1031800020932C01260F371F30938B0120938A0147
:103190006CE271E087E690E00E94A9166AE871E0AF
:1031A0008AE690E00E94A9166CE871E08DE690E056
:1031B0000E94A916809131058330D1F50E94A8079D
:1031C00060E080E00E94AC098CE293E00E94610A1A
:1031D00080915F0590916005909393018093920197
:1031E00020918C0130918D01821B930B63E070E084
:1031F0000E94F434260F371F30938F0120938E01E5
:10320000260F371F30939101209390016EE871E0F3
:1032100080E790E00E94A91660E971E083E790E002
:103220000E94A91662E971E086E790E00E94A91663
:10323000809131058430D1F50E94A80760E080E0DC
:103240000E94AC098DE393E00E94610A80915F05C2
:10325000909160059093990180939801209192013B
:1032600030919301821B930B63E070E00E94F43471
:10327000260F371F3093950120939401260F371F97
:10328000309397012093960164E971E089E790E01B
:103290000E94A91666E971E08CE790E00E94A916E9
:1032A00068E971E08FE790E00E94A91680913105EE
:1032B000853009F048C00E94A80760E080E00E94C5
:1032C000AC098EE493E00E94610A80915F059091C1
:1032D00060059093A1018093A00120919801309105
:1032E0009901821B930B97FD03969595879595956C
:1032F0008795280F391F30939B0120939A01280F3F
:10330000391F30939D0120939C01820F931F90934E
:103310009F0180939E016AE971E082E890E00E943B
:10332000A9166CE971E085E890E00E94A9166EE9A3
:1033300071E088E890E00E94A91660EA71E08BE8ED
:1033400090E00E94A91680913105863009F048C0AE
:103350000E94A80760E080E00E94AC098FE593E03E
:103360000E94610A80915F05909160059093A90188
:103370008093A8012091A0013091A101821B930BA1
:1033800097FD03969595879595958795280F391FF5
:103390003093A3012093A201280F391F3093A50178
:1033A0002093A401820F931F9093A7018093A601FD
:1033B00062EA71E08EE890E00E94A91664EA71E08A
:1033C00081E990E00E94A91666EA71E084E990E044
:1033D0000E94A91668EA71E087E990E00E94A916A8
:1033E00080913105873009F048C00E94A80760E04D
:1033F00080E00E94AC0980E793E00E94610A80911E
:103400005F05909160059093B1018093B001209188
:10341000A8013091A901821B930B97FD0396959506
:10342000879595958795280F391F3093AB01209389
:10343000AA01280F391F3093AD012093AC01820FF0
:10344000931F9093AF018093AE016AEA71E08AE91D
:1034500090E00E94A9166CEA71E08DE990E00E946C
:10346000A9166EEA71E080EA90E00E94A91660EB6E
:1034700071E083EA90E00E94A9160E94A906609379
:103480006105709362058093630590936405809154
:103490008805909189050A9724F010928905109269
:1034A0008805DF91CF911F910F910C940015AF9279
:1034B000BF92CF92DF92EF92FF920F931F93CF9321
:1034C000DF9300D0CDB7DEB78B016B0124E0C20ED5
:1034D000D11C7B015C01A61AB70AC5018E0D9F1D88
:1034E0009A838983F70161917F01CE0101960E9441
:1034F000BE14EC14FD0489F7C8010F900F90DF9102
:10350000CF911F910F91FF90EF90DF90CF90BF90E0
:10351000AF9008950F931F93CF93DF9300D0CDB753
:10352000DEB78B019A838983FB016081CE0101960E
:103530000E94BE14C8010F900F90DF91CF911F9190
:103540000F9108958F929F92AF92BF92FF920F9327
:103550001F93CF93DF93EC01F090860500918805CF
:1035600010918905F11052C00230110509F44EC0C6
:103570008130910509F0B6C0809131058F5F8730A9
:1035800008F0AEC0809331054091840150918501CF
:1035900060918601709187018091C0019091C10175
:1035A000A091C201B091C301840F951FA61FB71F40
:1035B0008093C0019093C101A093C201B093C30155
:1035C0006091C0017091C1018091C2019091C301CD
:1035D00020918401309185014091860150918701AD
:1035E0008090840190908501A0908601B090870121
:1035F0000E940835C501B4010E94E4346093C00103
:103600007093C1018093C2019093C3018091C00166
:103610009091C101A091C201B091C3018138944A37
:10362000AF4BB74060F080E894EAAFEBB7E080932F
:10363000C0019093C101A093C201B093C3018091D6
:10364000C0019091C101A091C201B091C301803A23
:103650009648A140B10560F480EA96E8A1E0B0E0A8
:103660008093C0019093C101A093C201B093C301A4
:1036700081E0F812BBC0C130D10509F082C0409191
:10368000840150918501609186017091870180913C
:10369000510590915205A0915305B0915405840FA6
:1036A000951FA61FB71F8093510590935205A093B5
:1036B0005305B09354050130110509F0D0C0809135
:1036C000730590917405A0917505B091760580936E
:1036D000C0019093C101A093C201B093C3019DC0EA
:1036E00087E050CF019609F091CF4091840150912D
:1036F000850160918601709187018091C001909150
:10370000C101A091C201B091C301841B950BA60B0E
:10371000B70B8093C0019093C101A093C201B093F5
:10372000C3016091C0017091C1018091C20190916B
:10373000C30120918401309185014091860150910F
:1037400087018090840190908501A0908601B090BF
:1037500087010E940835C501B4010E94E4346093DA
:10376000C0017093C1018093C2019093C301809105
:1037700031058150823018F08093310547CF81E0C8
:10378000FBCFCF3FDC0709F0B7C2409184015091D5
:10379000850160918601709187018091510590911A
:1037A0005205A0915305B0915405841B950BA60BAF
:1037B000B70B8093510590935205A0935305B09396
:1037C00054050130110509F04AC0809173059091AC
:1037D0007405A0917505B09176058093C001909312
:1037E000C101A093C201B093C301BDC10130110555
:1037F000B1F58091730590917405A0917505B09114
:1038000076058093C0019093C101A093C201B0934B
:10381000C301C130D10509F0A2C14091840150918A
:1038200085016091860170918701809134019091AA
:103830003501A0913601B0913701840F951FA61F65
:10384000B71F8093340190933501A0933601B09354
:10385000370164E371E08AE190E00E94571A809199
:103860008805909189050297E9F5809173059091FB
:103870007405A0917505B09176058093C001909371
:10388000C101A093C201B093C301C130D10509F0B9
:103890007FC18091B6019091B701A091B801B0911C
:1038A000B901813A22E0920724E9A207B105A4F404
:1038B000409184015091850160918601709187014A
:1038C000840F951FA61FB71F8093B6019093B70171
:1038D000A093B801B093B90166EB71E085E190E087
:1038E0000E94571A80918805909189050397E9F500
:1038F0008091730590917405A0917505B09176053E
:103900008093C0019093C101A093C201B093C30101
:10391000C130D10509F05DC18091BB019091BC011E
:10392000A091BD01B091BE01813A22E0920724E945
:10393000A207B105A4F440918401509185016091E2
:10394000860170918701840F951FA61FB71F809372
:10395000BB019093BC01A093BD01B093BE016BEB82
:1039600071E082E090E00E94571A80918805909162
:103970008905049719F58091730590917405A091BC
:103980007505B09176058093C0019093C101A09315
:10399000C201B093C301C130D10509F03BC168EA4F
:1039A00072E080EB96E00E94A31481E08093BF0157
:1039B0006FEB71E090E080E00E948A1A80918805A8
:1039C00090918905059719F580917305909174057B
:1039D000A0917505B09176058093C0019093C101C7
:1039E000A093C201B093C301C130D10509F01FC13A
:1039F00068EA72E08AEA96E00E94A31481E080936C
:103A0000BA016AEB71E08DE090E00E948A1A809121
:103A10008805909189050697B1F58091730590917D
:103A20007405A0917505B09176058093C0019093BF
:103A3000C101A093C201B093C301C130D10509F007
:103A400003C140918401509185016091860170917C
:103A5000870180916F0590917005A0917105B091DB
:103A60007205840F951FA61FB71F80936F05909353
:103A70007005A0937105B09372056FE675E084E25E
:103A800090E00E94571A80918805909189050797C8
:103A9000B9F58091730590917405A0917505B09169
:103AA00076058093C0019093C101A093C201B093A9
:103AB000C301C130D10509F0E5C08091300190917A
:103AC0003101A0913201B0913301805F984DAF4F29
:103AD000BF4F803823EC920729ECA20721E0B20700
:103AE0000CF0CBC08093300190933101A093320150
:103AF000B093330160E371E088E290E00E94571ACE
:103B000080918805909189058830910509F0D8C089
:103B10008091730590917405A0917505B09176051B
:103B20008093C0019093C101A093C201B093C301DF
:103B300064E972E0CF3FDC0729F0219709F0D2C099
:103B400068EA72E084EA96E0DF91CF911F910F91CD
:103B5000FF90BF90AF909F908F900C94A314CF3F95
:103B6000DC0709F076CE4091840150918501609187
:103B70008601709187018091340190913501A09167
:103B80003601B0913701841B950BA60BB70B59CEAC
:103B9000CF3FDC0709F0A0CE8091B6019091B7012C
:103BA000A091B801B091B901813A26E8920721E0CD
:103BB000A207B1050CF490CE40918401509185018B
:103BC0006091860170918701841B950BA60BB70B42
:103BD0007BCECF3FDC0709F0C2CE8091BB01909134
:103BE000BC01A091BD01B091BE01813A26E89207C7
:103BF00021E0A207B1050CF4B2CE409184015091AE
:103C000085016091860170918701841B950BA60B3D
:103C1000B70B9DCECF3FDC0709F0CACE64E972E056
:103C200080EB96E00E94A3141092BF01C1CECF3F5B
:103C3000DC0709F0E6CE64E972E08AEA96E00E94C9
:103C4000A3141092BA01DDCECF3FDC0709F015CFE7
:103C500040918401509185016091860170918701A6
:103C600080916F0590917005A0917105B0917205DA
:103C7000841B950BA60BB70BF8CE80E893ECA9EC50
:103C8000B1E030CFCF3FDC0709F034CF8091300175
:103C900090913101A0913201B0913301805197424E
:103CA000A109B109813026E392072EE6A20721E09F
:103CB000B2070CF017CF80E096E3AEE6B1E012CF8A
:103CC000099781F48091730590917405A091750511
:103CD000B09176058093C0019093C101A093C20179
:103CE000B093C301DF91CF911F910F91FF90BF90CF
:103CF000AF909F908F9008950130110509F0AFCDDE
:103D00008091730590917405A0917505B091760529
:103D10008093C0019093C101A093C201B093C301ED
:103D200098CD1F920F920FB60F9211242F933F93AD
:103D30004F935F936F937F938F939F93AF93BF93B3
:103D4000EF93FF938BEF95E00E94C304FF91EF91F7
:103D5000BF91AF919F918F917F916F915F914F91A3
:103D60003F912F910F900FBE0F901F9018951F92AB
:103D70000F920FB60F9211242F938F939F93EF936F
:103D8000FF93E0910B06F0910C068081E091110603
:103D9000F091120682FD1BC09081809114068F5F06
:103DA0008F7320911506821741F0E0911406F0E020
:103DB000E550FA4F958F80931406FF91EF919F91F4
:103DC0008F912F910F900FBE0F901F9018958081AB
:103DD000F4CF1F920F920FB60F9211242F933F939F
:103DE0008F939F93AF93BF9380912005909121056E
:103DF000A0912205B091230530911F0523E0230FE8
:103E00002D3758F50196A11DB11D20931F058093F4
:103E1000200590932105A0932205B093230580915E
:103E2000240590912505A0912605B09127050196BE
:103E3000A11DB11D8093240590932505A09326050F
:103E4000B0932705BF91AF919F918F913F912F9193
:103E50000F900FBE0F901F90189526E8230F029623
:103E6000A11DB11DD2CF1F920F920FB60F92112438
:103E70002F933F934F935F936F937F938F939F9372
:103E8000AF93BF93EF93FF938091B900887F803603
:103E900009F44AC0F0F5883209F4A7C018F580315A
:103EA00009F49BC0B8F4882309F4F9C0883009F4F8
:103EB00094C0FF91EF91BF91AF919F918F917F91AE
:103EC0006F915F914F913F912F910F900FBE0F9087
:103ED0001F901895883109F488C0803251F780937B
:103EE000D40514C0803409F49DC040F48033B9F384
:103EF0008833F9F68093D40585ECB0C0803509F499
:103F000085C0883509F496C0883499F60E94B506B4
:103F1000D0CF883909F48CC038F5883729F050F4AF
:103F2000883611F0803729F683E08093D605109209
:103F30001E0557C0883809F47BC0803919F08038D5
:103F400009F0B7CF80911E05803208F071C0E09172
:103F50001E0581E08E0F80931E058091BB00F0E06E
:103F6000E250FB4F80833DC0803B39F0E0F4803A63
:103F700009F479C0883A09F09CCF84E08093D60593
:103F80001092FD041092FC04E0918C05F0918D05D7
:103F900009958091FC0481110FC081E08093FC049D
:103FA0001092DC0409C0803C09F4A6CF883C09F4D7
:103FB000A3CF883B09F07DCFE091FD0481E08E0F17
:103FC0008093FD04F0E0E452FB4F80818093BB00BE
:103FD0009091FD048091FC0429C08091B1058093EB
:103FE000BB0085EC8093BC0064CF9091D305809199
:103FF000D205981758F5E091D30581E08E0F809394
:10400000D305F0E0EE54FA4F8081E9CFE091D3057B
:1040100081E08E0F8093D3058091BB00F0E0EE54D9
:10402000FA4F80839091D3058091D2059817C8F2FA
:1040300085E8D8CFE091D30581E08E0F8093D3053A
:104040008091BB00F0E0EE54FA4F80838091D5055B
:1040500081115CCF81E08093B00584EA8093BC003D
:104060001092D60526CF85EC8093BC001092D60521
:1040700080911E05803230F4E0911E05F0E0E250A0
:10408000FB4F108260911E0570E0E0918A05F0916F
:104090008B058EEF94E0099510921E050ACF1092C1
:1040A000D40534CF1F920F920FB60F921124CF92E6
:1040B000DF92EF92FF920F931F932F933F934F93B3
:1040C0005F936F937F938F939F93AF93BF93CF93A0
:1040D000DF93EF93FF938091DC060E947B05EC0158
:1040E0008091DB060E947B059091DA069F70CC0FD1
:1040F000DD1FC82B24E0929FC001112486539E4FE0
:10410000C80FD92FD11DC881C093DA06C07361F1E1
:104110000E94A906009128051091290520912A05E1
:1041200030912B056B017C01C01AD10AE20AF30A17
:104130009701860100932D0510932E0520932F05DE
:1041400030933005609328057093290580932A05E4
:1041500090932B0581E090E0C03121F0C03221F432
:104160008FEF9FEF0E94A21AFF91EF91DF91CF9105
:10417000BF91AF919F918F917F916F915F914F917F
:104180003F912F911F910F91FF90EF90DF90CF9073
:104190000F900FBE0F901F901895CF93DF93EBEF0A
:1041A000F5E01382128288EE93E0A0E0B0E0848311
:1041B0009583A683B7832AEE31E03183208325ECF3
:1041C00030E03587248724EC30E03787268720ECE1
:1041D00030E0318B208B21EC30E0338B228B22ECD2
:1041E00030E0358B248B26EC30E0378B268B118E1C
:1041F000128E138E148EE8E9F6E013821282848305
:104200009583A683B7838CEF91E091838083EBE164
:10421000F7E0138212828EE092E09183808389E03E
:1042200084838FEF8583C8E0C68387E0878386E039
:10423000808785E0818784E08287138614861586CF
:104240001686178681E00E940609EDEDF6E0C0AF04
:10425000C1AF11AA12AA13AA118612861386148658
:10426000158616861786108A118A128A138A148A6E
:10427000158A168A178A108E118E128E138E148E3E
:10428000158E168E178E10A211A212A213A214A2BE
:1042900015A216A217A210A611A612A613A614A65E
:1042A00015A616A617A610AA80ED90E9A7EFB1E013
:1042B00082AF93AFA4AFB5AFCAEDD6E083E08983F8
:1042C00082E08A8360E083E00E94040660E08A81E5
:1042D0000E94040661E089810E94A40561E08A8150
:1042E0000E94A405188261E873E084ED96E00E94C4
:1042F000AD1463E873E08EEC96E00E94AD1468E8BC
:1043000073E088EC96E00E94AD1464E674E082EC01
:1043100096E00E94AD1464E674E08CEB96E00E9497
:10432000AD1464E674E086EB96E00E94AD1468EA92
:1043300072E080EB96E00E94AD1468EA72E08AEACF
:1043400096E00E94AD1464E972E084EA96E0DF91A1
:10435000CF910C94AD14CF93DF93CDB7DEB7A79771
:104360000FB6F894DEBF0FBECDBF789484B58260DF
:1043700084BD84B5816084BD85B5826085BD85B509
:10438000816085BD80916E00816080936E00109287
:104390008100809181008260809381008091810002
:1043A0008160809381008091800081608093800093
:1043B0008091B10084608093B1008091B0008160F1
:1043C0008093B00080917A00846080937A0080911D
:1043D0007A00826080937A0080917A008160809375
:1043E0007A0080917A00806880937A001092C100F0
:1043F000E0910B06F0910C0682E08083E0910706C5
:10440000F09108061082E0910906F0910A068FECFF
:10441000808310921306E0910F06F091100686E05B
:104420008083E0910D06F0910E068081806180838B
:10443000E0910D06F0910E06808188608083E09106
:104440000D06F0910E06808180688083E0910D0654
:10445000F0910E0680818F7D808382E00E940609A4
:1044600081E00E9400098BE39FE10197F1F70E9430
:10447000D20561E08AE00E94040661E08BE00E94C0
:10448000040661E08CE00E94040661E08DE00E9479
:10449000040660E08FE00E94040661E080E10E9473
:1044A000040661E081E10E94040668E671E081E0B3
:1044B0000E94C10960E671E082E00E94C10968E5DE
:1044C00071E083E00E94C10960E571E084E00E9430
:1044D000C10968E471E085E00E94C10960E471E00F
:1044E00086E00E94C10968E371E087E00E94C1098B
:1044F0006CE275E089E090E00E941714DC018C9179
:104500008D3909F4B4C76FEB71E090E080E00E9450
:104510008A1A6BEB71E082E090E00E94571A6BE719
:1045200075E088E090E00E948A1A8DE990E09A8315
:104530008983BE016F5F7F4F89E090E00E94A916DA
:104540006AEB71E08DE090E00E948A1A61E575E007
:104550008FE090E00E94571A66EB71E085E190E0F1
:104560000E94571A64E371E08AE190E00E94571AB2
:104570008FE190E00E94D7146BE675E084E290E052
:104580000E94571A60E371E088E290E00E94571A97
:1045900068E871E087E390E00E94A91660E871E0A6
:1045A0008CE390E00E94571A6CE771E081E490E0A0
:1045B0000E94571A68E771E086E490E00E94571A5B
:1045C00064E771E08BE490E00E94571A60E771E0C5
:1045D00080E590E00E94571A6EE271E084E690E078
:1045E0000E94A9166CE271E087E690E00E94A9168D
:1045F0006AE871E08AE690E00E94A9166CE871E032
:104600008DE690E00E94A9166EE871E080E790E0E8
:104610000E94A91660E971E083E790E00E94A91664
:1046200062E971E086E790E00E94A91664E971E012
:1046300089E790E00E94A91666E971E08CE790E0B6
:104640000E94A91668E971E08FE790E00E94A91620
:104650006AE971E082E890E00E94A9166CE971E0D5
:1046600085E890E00E94A9166EE971E088E890E084
:104670000E94A91660EA71E08BE890E00E94A916FA
:1046800062EA71E08EE890E00E94A91664EA71E0A7
:1046900081E990E00E94A91666EA71E084E990E061
:1046A0000E94A91668EA71E087E990E00E94A916C5
:1046B0006AEA71E08AE990E00E94A9166CEA71E06A
:1046C0008DE990E00E94A9166EEA71E080EA90E020
:1046D0000E94A91660EB71E083EA90E00E94A9169F
:1046E00068E271E08AEA90E00E94571A64E271E0A1
:1046F0008FEA90E00E94571A60E271E084EB90E04C
:104700000E94571A6CE171E089EB90E00E94571A01
:1047100068E171E08EEB90E00E94571A64E171E06D
:1047200083EC90E00E94571A60E171E088EC90E021
:104730000E94571A6CE071E08DEC90E00E94571ACD
:1047400068E071E082ED90E00E94571A64E071E049
:1047500087ED90E00E94571A6FEB71E090E080E0E7
:104760000E941714DC018C918093BF016BEB71E008
:1047700082E090E00E942A13FC0180819181A28155
:10478000B3818093BB019093BC01A093BD01B09312
:10479000BE016BE775E088E090E00E941714DC0131
:1047A0008C9180937B0567E675E085E190E00E943F
:1047B0002A13FC0180819181A281B3818093B6018B
:1047C0009093B701A093B801B093B9016AEB71E07F
:1047D0008DE090E00E941714DC018C918093BA0167
:1047E00061E575E08FE090E00E942A13FC01808172
:1047F0009181A281B3818093510590935205A0933A
:104800005305B093540564E371E08AE190E00E949F
:104810002A13FC0180819181A281B38180933401AC
:1048200090933501A0933601B09337018FE190E06A
:104830000E9465338093000180E290E00E9465331E
:104840008093010181E290E00E9465338093020130
:1048500082E290E00E946533809303018091000121
:1048600090910101A0910201B09103018093C001D8
:104870009093C101A093C201B093C3016FE675E0AC
:1048800084E290E00E942A13FC0180819181A28140
:10489000B38180936B0590936C05A0936D05B093E5
:1048A0006E0560E371E088E290E00E942A13FC014B
:1048B00080819181A281B3818093300190933101F5
:1048C000A0933201B093330168E871E087E390E090
:1048D0000E941613DC018D919C9190938901809325
:1048E000880160E871E08CE390E00E942A13FC01EB
:1048F00080819181A281B381809380019093810115
:10490000A0938201B09383016CE771E081E490E0B1
:104910000E942A13FC0180819181A281B38180933E
:104920007C0190937D01A0937E01B0937F0168E7A5
:1049300071E086E490E00E942A13FC01808191815D
:10494000A281B3818093780190937901A0937A0139
:10495000B0937B0164E771E08BE490E00E942A133E
:10496000FC0180819181A281B38180937401909335
:104970007501A0937601B093770160E771E080E55F
:1049800090E00E942A13FC0180819181A281B38171
:104990008093700190937101A0937201B0937301A1
:1049A0008091340190913501A0913601B091370189
:1049B0008093110790931207A0931307B0931407E5
:1049C000C0903001D0903101E0903201F09033017D
:1049D0000E94D20562E987EB0E946507C114D104E9
:1049E000E104F104D1F08FE00E94CA07682F6F73D1
:1049F000F1E8CF16F3ECDF06F9ECEF06F1E0FF0685
:104A000008F044C5C0921707D0921807E092190722
:104A1000F0921A078FE00E94650760E880E10E942B
:104A2000650760E881E10E94650760E882E10E9415
:104A300065076CE080E10E9465076CE081E10E94FF
:104A400065076CE082E10E94650760E281EB0E94ED
:104A5000650760E881EB0E94650710E000E020E058
:104A600034E04BE654EF64E170E080E090E00E94B7
:104A7000330D61E081E090E00E943D0890E080E02D
:104A80000E94310881E090E00E94310882E090E0CD
:104A90000E94310861E873E084ED96E00E94A3145F
:104AA00062E08EE00E94040680916800846080933A
:104AB000680080916D008C6080936D0078940E94F6
:104AC000A906609328057093290580932A05909381
:104AD0002B0588EE93E0A0E0B0E080932D05909345
:104AE0002E05A0932F05B093300510917B05113052
:104AF00061F46CE873E08EEC96E00E94A3141093CE
:104B0000650561E080E10E94A40580917B0581112B
:104B10000CC063E873E08EEC96E00E94A314109240
:104B2000650560E080E10E94A40590913A058091BE
:104B300085059111E1C4883208F07DC08091360569
:104B40008130A9F460E871E08CE390E00E942A13C0
:104B5000FC0180819181A281B3818093C0019093F7
:104B6000C101A093C201B093C30110923605809198
:104B700035058130A9F46CE771E081E490E00E9492
:104B80002A13FC0180819181A281B3818093C001AD
:104B90009093C101A093C201B093C3011092350557
:104BA000809134058130A9F468E771E086E490E0F3
:104BB0000E942A13FC0180819181A281B38180939C
:104BC000C0019093C101A093C201B093C3011092A0
:104BD0003405809133058130A9F464E771E08BE4FA
:104BE00090E00E942A13FC0180819181A281B3810F
:104BF0008093C0019093C101A093C201B093C301FF
:104C000010923305809132058130A9F460E771E09C
:104C100080E590E00E942A13FC0180819181A281AD
:104C2000B3818093C0019093C101A093C201B0935E
:104C3000C30110923205809185058150873260F45E
:104C400080913A05813041F460E080E00E94AC0937
:104C500081E993E00E94610A80918505883260F0C5
:104C600080913A05813041F460E080E00E94AC0917
:104C700086E993E00E94610A80913A05811102C0A1
:104C80001092850580913D0590913E05019709F0B0
:104C900098C080912D0590912E05A0912F05B0917F
:104CA000300585369105A105B105C0F02AE030E058
:104CB00040E050E0209384013093850140938601C9
:104CC000509387018EE690E0A0E0B0E080932D0540
:104CD00090932E05A0932F05B093300580912D055C
:104CE00090912E05A0912F05B09130054F97A10905
:104CF000B10986349105A105B105C0F422E330E085
:104D000040E050E020938401309385014093860178
:104D10005093870181E490E0A0E0B0E080932D05FE
:104D200090932E05A0932F05B093300580912D050B
:104D300090912E05A0912F05B09130050697A109FD
:104D4000B1094997A105B105C0F424E630E040E07F
:104D500050E0209384013093850140938601509365
:104D6000870181E190E0A0E0B0E080932D05909371
:104D70002E05A0932F05B093300580912D059091BD
:104D80002E05A0912F05B09130050697A105B1051C
:104D9000C0F428EE33E040E050E0209384013093EB
:104DA000850140938601509387018FE090E0A0E059
:104DB000B0E080932D0590932E05A0932F05B0931E
:104DC00030058091880590918905892BB1F560E0C7
:104DD00084E00E94AC098091C0019091C101A09132
:104DE000C201B091C3018093450590934605A093FD
:104DF0004705B09348056091C0017091C101809151
:104E0000C2019091C30120E432E44FE050E00E94DF
:104E10000835209341053093420540934305509354
:104E200044050E94630A60E08FE00E94AC0964EDD3
:104E300076E08BE197E00E9437048EE00E94400606
:104E40008EE00E9440067C0190933C0580933B05D8
:104E50006AE070E080E090E00E9477068EE00E94B9
:104E600040068EE00E944006092E000CAA0BBB0BE8
:104E7000A7010F2C000C660B770B4C015D01E3E0E2
:104E80008E1A9108A108B108481559056A057B05D5
:104E900064F00396A11DB11D84179507A607B707F7
:104EA00024F0F0925005E0924F05E0904F05F0900D
:104EB0005005F5E8EF16F3E0FF060CF465C3109219
:104EC0003A0580913905811106C060E081E10E94B8
:104ED000A40510928705809188019091890100971F
:104EE00009F0FBC421E030E030933E0520933D05FE
:104EF00024EF31E040E050E08530910509F014C521
:104F0000209384013093850140938601509387015B
:104F100010923E0510923D0580918805909189057B
:104F20001816190614F40E94D01680918705813056
:104F3000B9F58091880590918905892B89F5E090D4
:104F40003F05F09040059FEFE91AF90AF0924005FD
:104F5000E0923F0584E10E944006BC01990F880B56
:104F6000990B0E9448322B013C0185E10E944006CA
:104F7000BC01990F880B990B0E9448324B015C01D0
:104F8000AC019B01C301B2010E94DA3487FD08C560
:104F900061E080E00E94AC098BE993E00E94610A25
:104FA00081E090918605913009F080E091E02091B8
:104FB0008705211190E0892309F4BFC080918805FD
:104FC00090918905892B09F0B8C08091B201909128
:104FD000B301A091B401B091B501803AE6E89E0713
:104FE000E1E0AE07B1050CF06CC58091C001909175
:104FF000C101A091C201B091C301805A9648A1405D
:10500000B109B095A095909581959F4FAF4FBF4F37
:105010008093510590935205A0935305B093540586
:1050200080914F059091500587599109C197D0F40F
:1050300080914D0590914E05843691059CF4019622
:1050400090934E0580934D05C29761F410925105DF
:1050500010925205109253051092540510924E056D
:1050600010924D050E94EF0A8091C0019091C101FC
:10507000A091C201B091C3014091510550915205D8
:105080006091530570915405840F951FA61FB71F9B
:105090008093B2019093B301A093B401B093B50192
:1050A0008091490590914A05A0914B05B0914C051E
:1050B000481759076A077B07B1F061E575E08FE093
:1050C00090E00E94571A8091510590915205A0914D
:1050D0005305B09154058093490590934A05A093D8
:1050E0004B05B0934C0561E084E00E94AC096091EF
:1050F000B2017091B3018091B4019091B5016093B8
:10510000450570934605809347059093480520E434
:1051100032E44FE050E00E942A352093410530935D
:10512000420540934305509344050E94630A80E280
:105130000E94DD0980E20E94DD098091870590913F
:105140008605892B09F0FCC080918805909189051E
:10515000892B09F0F5C064E674E08CEB96E00E94C0
:10516000A3140E94A8070E94A9060E94A906C09045
:105170006105D0906205E0906305F09064056C19BC
:105180007D098E099F09643671058105910540F4FA
:1051900080915F059091600590935E0580935D0519
:1051A0000E94A9066C197D098E099F096436710554
:1051B0008105910598F00E94A9066C197D098E0958
:1051C0009F09683C71058105910540F480915F0558
:1051D0009091600590935C0580935B050E94A90601
:1051E0006C197D098E099F09683C7105810591053F
:1051F00098F00E94A9066C197D098E099F096C32EE
:1052000071408105910540F480915F0590916005A2
:1052100090935A05809359050E94A9066C197D093F
:105220008E099F096C3271408105910598F00E94AA
:10523000A9066C197D098E099F09603971408105A5
:10524000910540F480915F05909160059093580519
:10525000809357050E94A9066C197D098E099F0944
:10526000603971408105910598F00E94A9066C197A
:105270007D098E099F09653F71408105910540F4C4
:1052800080915F0590916005909356058093550538
:105290000E94A9066C197D098E099F09653F71401E
:1052A0008105910508F44AC080915D0590915E05E5
:1052B00020915B0530915C05820F931F2091590569
:1052C00030915A05820F931F209157053091580550
:1052D000820F931F2091550530915605820F931F21
:1052E00065E070E00E94F4347B0170936005609388
:1052F0005F0560EB71E083EA90E00E941613FC0109
:1053000080819181E816F9060CF4F2C38CEB93E0EE
:105310000E94751461E084E00E94AC096CEB76E0B9
:105320008BE197E00E9437040E94A9066093610513
:105330007093620580936305909364050E94EF0A61
:105340006FE675E084E290E00E942A13FC01808100
:105350009181A281B38180936B0590936C05A0939A
:105360006D05B0936E0567E675E085E190E00E94FB
:105370002A13FC0180819181A281B3818093B601BF
:105380009093B701A093B801B093B901F09087054D
:10539000F1E0FF1210C08091C0019091C101A09175
:1053A000C201B091C3018093B2019093B301A09365
:1053B000B401B093B5018091C0019091C101A09159
:1053C000C201B091C30180389649A849B10508F4DB
:1053D0002FC5809166058111CBC461E873E084ED2F
:1053E00096E00E94A31468E873E088EC96E00E94BF
:1053F000A31480918605813009F0AFC48091B20179
:105400009091B301A091B401B091B5014091B60162
:105410005091B7016091B8017091B901841B950B4F
:10542000A60BB70B8093810590938205A09383050B
:10543000B093840580916505813009F03EC531E067
:10544000F3123BC58091810590918205A09183055F
:10545000B091840540916B0550916C0560916D058C
:1054600070916E05841B950BA60BB70BCDC48EE017
:105470000E944006853F91400CF46EC98EE00E9468
:1054800040068A3892400CF43EC866C9D701C6016E
:105490008158934CA94CB1408038934CA94CB140F1
:1054A00070F4F694E794D794C794C0921707D092FB
:1054B0001807E0921907F0921A076064ABCAD70187
:1054C000C60181509748A349B34081159A45A24629
:1054D000B24008F09FCA82E0F694E794D794C7944C
:1054E0008A95D1F7C0921707D0921807E092190752
:1054F000F0921A0760688ECA913009F09CCB88320E
:1055000051F480913605813031F48CE390E00E94B3
:10551000D7141092360580918505883251F4809118
:105520003505813031F481E490E00E94D714109267
:10553000350580918505883251F48091340581309C
:1055400031F486E490E00E94D714109234058091E3
:105550008505883251F480913305813031F48BE434
:1055600090E00E94D714109233058091850588320F
:1055700009F061CB80913205813009F06DCB80E577
:1055800090E00E94D71455CB28E4E216F1046CF4A5
:1055900080913A05811109C061E081E10E94A40572
:1055A00081E08093870580933A05C701895491096A
:1055B0008D34910538F580913A05811123C0809191
:1055C000390581110BC061E081E10E94A40581E0F1
:1055D000809339058093870580933A0580913A0539
:1055E000811179CC10913905113009F074CC60E04B
:1055F00081E10E94A405109239051092870510934D
:105600003A0569CCC701875991098034910508F59D
:1056100080913A0581111DC080918605811109C0D4
:1056200081E08093860580933A0510924E05109292
:105630004D0580913A0581110CC08091860581301D
:1056400041F41092860580933A0510924E0510920F
:105650004D05C701885D9109C697D8F480913A0538
:10566000811117C0809137059091380501968A30D5
:1056700091052CF4909338058093370504C010925F
:1056800038051092370581E080933A050E94501347
:1056900022CCC7018F509140C19770F480913A0598
:1056A00081110AC08091370590913805019797FFC5
:1056B000E1CF89E090E0DECFC701815491408C9723
:1056C000C0F580913A05811134C080916505811142
:1056D00011C061E080E10E94A40511E010937B05F8
:1056E0006CE873E08EEC96E00E94A31410936505BD
:1056F00010933A0580913A05811114C01091650507
:10570000113081F460E080E10E94A40510927B05D5
:1057100063E873E08EEC96E00E94A3141092650596
:1057200010933A056BE775E088E090E00E948A1AD2
:10573000D2CBC7018E5691408297D8F480913A051A
:10574000811117C080916605811105C081E08093A9
:10575000660580933A0580913A058111BCCB809112
:105760006605813009F0B7CB1092660580933A0543
:10577000B2CBC701815991408297F8F480913A05E4
:1057800081111BC080918801909189010196893017
:1057900091052CF4909389018093880104C01092A4
:1057A00089011092880181E080933A0568E871E0F0
:1057B00087E390E00E94A9168ECBC701845B9140DD
:1057C0004C9770F480913A0581110AC0809188014C
:1057D00090918901019797FFDDCF88E090E0DACFC3
:1057E0009701215D31402337310508F051C0809188
:1057F0008505803508F04CC08F5F8093850581E07A
:1058000080933A052931310558F48093360510927A
:1058100035051092340510923305109232055BCB9A
:1058200097012B5E31402931310528F4109236055D
:1058300080933505EECF9701255032402631310552
:1058400038F4109236051092350580933405E3CF75
:1058500097012C5132402431310548F4109236051D
:10586000109235051092340580933305D6CF9701F9
:10587000215332402331310558F4109236051092ED
:10588000350510923405109233058093320523CBF1
:1058900035E4E31A32E0F30A45E4E416F10408F0D3
:1058A0001ACB80913A05811116CB80918805909191
:1058B00089050196909389058093880521E02093BE
:1058C00031050A9724F0109289051092880581E02D
:1058D00080933A050E94D016FECA8130910589F462
:1058E00021E030E040E050E02093840130938501D6
:1058F000409386015093870110923E0510923D051A
:10590000F7CA82309105C1F42AE030E040E050E06F
:105910002093840130938501409386015093870141
:1059200010923E0510923D0586309105C1F488EE37
:1059300093E0A0E0B0E023C083309105C1F422E3FE
:1059400030E040E050E020938401309385014093A3
:1059500086015093870110923E0510923D058730D5
:105960009105B1F420E137E240E050E0C9CA84304B
:10597000910509F0BDCA84E690E0A0E0B0E0809314
:10598000840190938501A0938601B0938701C0CADA
:10599000089709F0C1CA80EA96E8A1E0B0E0EFCF2D
:1059A000A4E1EA16F1040CF4FBCA1092400510922F
:1059B0003F05A5019401C301B2010E94CD336B01E3
:1059C0007C01A3019201C501B4010E94CC339B016B
:1059D000AC01C701B6010E9439346B017C0120E0A3
:1059E00030E0A9010E94DA34181624F0F7FAF09496
:1059F000F7F8F09420E030E040EA50E4C501B4014B
:105A00000E94A73220E030EC4FE754E40E94393482
:105A10002CE238E540EB5CE30E9439349B01AC0199
:105A20000E94A73220E030E048E452E40E9439347A
:105A30004B015C0120E030E040E050E4C701B601DA
:105A40000E94CD332B013C01A701960160E070E07C
:105A500080E89FE30E9439349B01AC01C301B2018D
:105A60000E94CD339B01AC0160E070E080E890E4DF
:105A70000E943934A50194010E94A7324B015C01B8
:105A800061E080E00E94AC098EEA93E00E94610A26
:105A900042E0C701B6010E949F0B61E088E00E94CE
:105AA000AC0983EB93E00E94610A61E08BE00E9405
:105AB000AC0940E0C501B4010E949F0B87EB93E065
:105AC0006DCA8138944AAF4BB7400CF4A9CA4091D3
:105AD000C0015091C1016091C2017091C30180E881
:105AE00094EAAFEBB7E0841B950BA60BB70B90CAFB
:105AF00060EB71E083EA90E00E941613DC018D9167
:105B00009C918E159F051CF489EC93E001CC6EEA04
:105B100071E080EA90E00E941613FC01808191817F
:105B20008E159F051CF486ED93E0F2CB6CEA71E0D4
:105B30008DE990E00E941613DC018D919C918E15E9
:105B40009F051CF483EE93E0E3CB6AEA71E08AE9F7
:105B500090E00E941613FC01808191818E159F05B3
:105B60001CF480EF93E0D4CB68EA71E087E990E021
:105B70000E941613DC018D919C918E159F051CF4DB
:105B80008DEF93E0C5CB66EA71E084E990E00E9476
:105B90001613FC01808191818E159F051CF48AE00B
:105BA00094E0B6CB64EA71E081E990E00E941613BC
:105BB000DC018D919C918E159F051CF487E194E08A
:105BC000A7CB62EA71E08EE890E00E941613FC0118
:105BD000808191818E159F051CF484E294E098CB1E
:105BE00060EA71E08BE890E00E941613DC018D9171
:105BF0009C918E159F051CF481E394E089CB6EE99E
:105C000071E088E890E00E941613FC018081918188
:105C10008E159F051CF48EE394E07ACB6CE971E05D
:105C200085E890E00E941613DC018D919C918E1501
:105C30009F051CF48BE494E06BCB6AE971E082E889
:105C400090E00E941613FC01808191818E159F05C2
:105C50001CF488E594E05CCB68E971E08FE790E0A4
:105C60000E941613DC018D919C918E159F051CF4EA
:105C700085E694E04DCB66E971E08CE790E00E9408
:105C80001613FC01808191818E159F051CF482E71B
:105C900094E03ECB64E971E089E790E00E9416133E
:105CA000DC018D919C918E159F051CF48FE794E08B
:105CB0002FCB62E971E086E790E00E941613FC01A9
:105CC000808191818E159F051CF48CE894E020CB97
:105CD00060E971E083E790E00E941613DC018D918A
:105CE0009C918E159F051CF489E994E011CB6EE818
:105CF00071E080E790E00E941613FC0180819181A1
:105D00008E159F051CF486EA94E002CB6CE871E0E6
:105D10008DE690E00E941613DC018D919C918E150A
:105D20009F051CF483EB94E0F3CA6AE871E08AE60D
:105D300090E00E941613FC01808191818E159F05D1
:105D40001CF480EC94E0E4CA6AE871E087E690E035
:105D50000E9416138BE992E0DBCA81116BCB809114
:105D6000C0019091C101A091C201B091C3014ECB7D
:105D7000813009F05DC06DEC74E084ED96E00E9426
:105D8000A3146FEC74E088EC96E00E94A314809159
:105D90008605813009F041C08091B2019091B30134
:105DA000A091B401B091B5014091B6015091B701F5
:105DB0006091B8017091B901840F951FA61FB71F9C
:105DC0008093810590938205A0938305B093840509
:105DD00080916505813009F070C041E0F4126DC01A
:105DE0008091810590918205A0918305B0918405F1
:105DF00040916B0550916C0560916D0570916E0539
:105E0000840F951FA61FB71F80938105909382056D
:105E1000A0938305B093840550C08111D9CF8091A0
:105E2000C0019091C101A091C201B091C301BCCF4A
:105E30008091C0019091C101A091C201B091C301B4
:105E400080389649A849B105C0F580916605811151
:105E500077C06DEC74E084ED96E00E94A31468E8CE
:105E600073E088EC96E00E94A3148091860581304F
:105E700009F05BC08091B2019091B301A091B4018F
:105E8000B091B5014091B6015091B7016091B80150
:105E90007091B901840F951FA61FB71F80938105CC
:105EA00090938205A0938305B09384058091650546
:105EB000813019F4F81609F493CF4091810550917F
:105EC0008205609183057091840580917D05909194
:105ED0007E05A0917F05B0918005481759076A0794
:105EE0007B0709F061C12091CC063091CD068091ED
:105EF000C6069091C7062817390709F055C1809149
:105F0000C8069091C9066091C2067091C3060097B9
:105F100009F439C16115710509F05DC0232B09F43D
:105F20003FC1FC01808190E039C18111BFCF8091D8
:105F3000C0019091C101A091C201B091C301A2CF53
:105F4000813009F0BACF61E873E084ED96E00E94F9
:105F5000A3146FEC74E088EC96E00E94A314809187
:105F60008605813029F58091B6019091B701A09105
:105F7000B801B091B9014091B2015091B301609163
:105F8000B4017091B501841B950BA60BB70B8093E0
:105F9000810590938205A0938305B0938405809139
:105FA0006505813009F089CF91E0F91286CF4ACAA0
:105FB0008111F5CF4091C0015091C1016091C201A2
:105FC0007091C3018091B6019091B701A091B80181
:105FD000B091B901D8CF0E94D438E0C09130E1F43B
:105FE000F1E0FF1219C08130B9F461E081E090E086
:105FF0000E943D086091BB017091BC018091BD0180
:106000009091BE0124E630E040E050E00E94A135CE
:1060100001E010E00E94E30E8091BF01813009F0A1
:10602000D0C0F110CEC080917B05813009F0C9C08D
:10603000C3C00E9485378AA19BA19093B706809325
:10604000B6068CA19DA19093B9068093B8068EA147
:106050009FA19093BB068093BA061BA21AA21DA211
:106060001CA24FC186EB96E00E94FF128AC163ED2D
:1060700074E0CE0101960E94AD144091BA06509191
:10608000BB066091B6067091B706CE0101960E94DC
:106090004914811104C0CE0101960E94FF1241E013
:1060A00050E066ED74E0CE0101960E944914811122
:1060B00004C0CE0101960E94FF12BE016F5F7F4FA8
:1060C0008BEF95E00E943704CE0101960E941113D8
:1060D00064E670E080E090E00E94770660918105C0
:1060E00070918205809183059091840524E630E0CB
:1060F00040E050E00E94B03510E000E00E94E30E66
:106100008091810590918205A0918305B0918405CD
:1061100080937D0590937E05A0937F05B0938005C5
:106120008091C0019091C101A091C201B091C301C1
:106130008093730590937405A0937505B0937605CD
:106140008091880590918905892B69F48091850556
:10615000811109C060E00E94AC096EEC76E08BE131
:1061600097E00E94370480E090E0892B11F40C94B2
:1061700095250E94AF04882311F40C9495250E9464
:1061800000000C9495256115710551F0232B41F009
:10619000DB018C9190E0919581959109892B21F4F7
:1061A00080917C058F1579F09091BF01992321F0A2
:1061B00080917B05811112CF60E081E090E00E9428
:1061C0003D08F0927C058091BA01811105C060E024
:1061D00082E090E00E943D088091BA018130A1F5F3
:1061E00061E082E090E00E943D086091B60170910C
:1061F000B7018091B8019091B901C0907705D09016
:106200007805E0907905F0907A056C157D058E058E
:106210009F05D1F024E630E040E050E00E94A13537
:1062200002E010E00E94E30E8091B6019091B70168
:10623000A091B801B091B90180937705909378054A
:10624000A0937905B0937A0540918105509182051C
:10625000609183057091840580917D0590917E0504
:10626000A0917F05B0918005481759076A077B0701
:1062700009F466CF8091880590918905892B09F0F2
:106280005FCF8FE190E00E94D7140E9400156091CB
:10629000C0017091C1018091C2019091C3011BA204
:1062A0001AA21DA21CA21FA21EA22AE0AE014F5FCD
:1062B0005F4F0E94F531BE016F5F7F4FCE01829626
:1062C0000E94A3148091B6069091B706009709F436
:1062D000B2CE6AA17BA16115710509F4AACE4091E5
:1062E000B8065091B9062EA13FA14217530708F4F2
:1062F000A0CE0E94DD388EA19FA19093BB06809313
:10630000BA061FA21EA2CE0182960E94111380918E
:10631000BA069091BB060B9708F0A9CE1BA21AA251
:106320001DA21CA21FA21EA24AE0BE016F5F7F4FEA
:1063300090E080E00E94EA31BE016F5F7F4FCE01A6
:1063400082960E94A3144091BA065091BB066091B8
:10635000B6067091B706CE0182960E94491481114B
:1063600004C0CE0182960E94FF126AA17BA1611532
:10637000710509F477CE4EA15FA186EB96E00E94ED
:106380008214CE0182960E941113C1CF84EA96E056
:106390000E9411138AEA96E00E94111380EB96E0A6
:1063A0000E94111386EB96E00E9411138CEB96E08D
:1063B0000E94111382EC96E00E94111388EC96E083
:1063C0000E9411138EEC96E00E94111384ED96E06A
:1063D0000C941113BB274A3031F4992322F4BDE207
:1063E000909581959F4F0C941832BB27FA01A62FE8
:1063F0006217710581059105330B30FB66F0AA2702
:10640000660F771F881F991FAA1FA21710F0A21BE3
:1064100063953850A9F7A05DAA3308F0A95DA19350
:1064200036F7B111B1931082CA010C943132BB27F7
:10643000FB015527AA27880F991FAA1FA41710F040
:10644000A41B83955051B9F7A05DAA3308F0A95D4C
:10645000A193009779F7B111B1931192CB010C94EC
:106460003132DC01FC01672F71917723E1F732971C
:1064700004C07C916D9370836291AE17BF07C8F31F
:1064800008950E94833208F481E00895E89409C0D9
:1064900097FB3EF490958095709561957F4F8F4F57
:1064A0009F4F9923A9F0F92F96E9BB279395F6956D
:1064B000879577956795B795F111F8CFFAF4BB0FEB
:1064C00011F460FF1BC06F5F7F4F8F4F9F4F16C04F
:1064D000882311F096E911C0772321F09EE8872FD9
:1064E000762F05C0662371F096E8862F70E060E095
:1064F0002AF09A95660F771F881FDAF7880F96950E
:10650000879597F90895990F0008550FAA0BE0E8B1
:10651000FEEF16161706E807F907C0F01216130665
:10652000E407F50798F0621B730B840B950B39F4A5
:106530000A2661F0232B242B252B21F408950A260B
:1065400009F4A140A6958FEF811D811D08950E9439
:10655000BA320C942B330E941D3338F00E9424333E
:1065600020F0952311F00C9414330C941A33112459
:106570000C945F330E943C3370F3959FC1F3950FE9
:1065800050E0551F629FF001729FBB27F00DB11DB7
:10659000639FAA27F00DB11DAA1F649F6627B00D47
:1065A000A11D661F829F2227B00DA11D621F739F30
:1065B000B00DA11D621F839FA00D611D221F749F3E
:1065C0003327A00D611D231F849F600D211D822F85
:1065D000762F6A2F11249F5750409AF0F1F08823AC
:1065E0004AF0EE0FFF1FBB1F661F771F881F9150D9
:1065F0005040A9F79E3F510580F00C9414330C9441
:106600005F335F3FE4F3983ED4F3869577956795C3
:10661000B795F795E7959F5FC1F7FE2B880F911D02
:106620009695879597F9089597F99F6780E870E0A8
:1066300060E008959FEF80EC089500240A941616F8
:10664000170618060906089500240A941216130660
:10665000140605060895092E0394000C11F48823EE
:1066600052F0BB0F40F4BF2B11F460FF04C06F5F0A
:106670007F4F8F4F9F4F089557FD9058440F551FE0
:1066800059F05F3F71F04795880F97FB991F61F0B4
:106690009F3F79F087950895121613061406551F2B
:1066A000F2CF4695F1DF08C0161617061806991F97
:1066B000F1CF86957105610508940895E894BB278C
:1066C00066277727CB0197F90895F999FECF92BDF8
:1066D00081BDF89A992780B50895262FF999FECFA4
:1066E0001FBA92BD81BD20BD0FB6F894FA9AF99AEF
:1066F0000FBE019608950E94BD33A59F900DB49FD3
:10670000900DA49F800D911D112408952F923F920A
:106710004F925F926F927F928F929F92AF92BF92B1
:10672000CF92DF92EF92FF920F931F93CF93DF935D
:10673000CDB7DEB7CA1BDB0B0FB6F894DEBF0FBEBA
:10674000CDBF09942A88398848885F846E847D8407
:106750008C849B84AA84B984C884DF80EE80FD8009
:106760000C811B81AA81B981CE0FD11D0FB6F8947F
:10677000DEBF0FBECDBFED010895A29FB001B39F54
:10678000C001A39F700D811D1124911DB29F700D3A
:10679000811D1124911D08955058BB27AA270E94DE
:1067A000E4330C942B330E941D3338F00E942433C1
:1067B00020F039F49F3F19F426F40C941A330EF4A8
:1067C000E095E7FB0C941433E92F0E943C3358F317
:1067D000BA17620773078407950720F079F4A6F5C6
:1067E0000C945E330EF4E0950B2EBA2FA02D0B0106
:1067F000B90190010C01CA01A0011124FF27591B06
:1068000099F0593F50F4503E68F11A16F040A22F0B
:10681000232F342F4427585FF3CF4695379527957C
:10682000A795F0405395C9F77EF41F16BA0B620B7B
:10683000730B840BBAF09150A1F0FF0FBB1F661FC2
:10684000771F881FC2F70EC0BA0F621F731F841F05
:1068500048F4879577956795B795F7959E3F08F02B
:10686000B0CF9395880F08F09927EE0F97958795ED
:1068700008950E944D340C942B330E94243358F019
:106880000E941D3340F029F45F3F29F00C9414332B
:1068900051110C945F330C941A330E943C3368F30B
:1068A0009923B1F3552391F3951B550BBB27AA27C9
:1068B00062177307840738F09F5F5F4F220F331F03
:1068C000441FAA1FA9F335D00E2E3AF0E0E832D0CB
:1068D00091505040E695001CCAF72BD0FE2F29D0CE
:1068E000660F771F881FBB1F261737074807AB07A0
:1068F000B0E809F0BB0B802DBF01FF2793585F4F15
:106900003AF09E3F510578F00C9414330C945F33A9
:106910005F3FE4F3983ED4F3869577956795B795F6
:10692000F7959F5FC9F7880F911D9695879597F901
:106930000895E1E0660F771F881FBB1F621773077A
:106940008407BA0720F0621B730B840BBA0BEE1F8F
:1069500088F7E09508950E94443388F09F5798F097
:10696000B92F9927B751B0F0E1F0660F771F881F54
:10697000991F1AF0BA95C9F714C0B13091F00E946E
:106980005E33B1E008950C945E33672F782F88272B
:10699000B85F39F0B93FCCF3869577956795B39595
:1069A000D9F73EF490958095709561957F4F8F4F04
:1069B0009F4F08950E94833208F48FEF08950E943C
:1069C0008332880B990B0895DB018F939F930E946C
:1069D0007B33BF91AF91A29F800D911DA39F900D1E
:1069E000B29F900D1124089597FB072E16F4009482
:1069F00007D077FD09D00E94CF3607FC05D03EF4C2
:106A0000909581959F4F0895709561957F4F08955A
:106A1000A1E21A2EAA1BBB1BFD010DC0AA1FBB1FA2
:106A2000EE1FFF1FA217B307E407F50720F0A21B14
:106A3000B30BE40BF50B661F771F881F991F1A9481
:106A400069F760957095809590959B01AC01BD01AB
:106A5000CF010895052E97FB1EF400940E94413546
:106A600057FD07D00E94083507FC03D04EF40C9464
:106A7000413550954095309521953F4F4F4F5F4F91
:106A8000089590958095709561957F4F8F4F9F4F9A
:106A90000895DF93CF931F930F939A9DF02D219F1D
:106AA000F00D8B9DF00D8A9DE02DF10D039FF00DF3
:106AB000029FE00DF11D4E9DE00DF11D5E9DF00D5C
:106AC0004F9DF00D7F936F93BF92AF925F934F9363
:106AD000D5010E94BD338B01AC01D7010E94BD33AB
:106AE000EB01E80FF91FD6010E9498352F913F91D5
:106AF000D6010E94BD33C60FD71FE81FF91FAF9103
:106B0000BF910E9498352F913F910E94BD33C60FCF
:106B1000D71FE81FF91FD6010E94BD33E60FF71FEC
:106B20009801BE01CF010F911F91CF91DF91089580
:106B30000E94BD33460F571FC81FD91F08F4319656
:106B4000089597FB57FF0C94B1359F938F930E9444
:106B5000B1356E1B7F0BAF91BF918A0B9B0B0895D4
:106B6000E894DF93CF93FC01DB010E94BD337F9358
:106B70006F93E9019A01AC01BF93AF933F932F93B9
:106B8000DF010E94BD3326F46C1B7D0B820B930B3F
:106B90009E01EB01FC010E949835AF91BF912F91AE
:106BA0003F910E949835BE01CF01F9012F913F918D
:106BB000CF91DF910895689401C0E894F92FF12BEB
:106BC00012F00C940F36A0E0B0E0E9EEF5E30C947F
:106BD0008C33092E059422F40E946B36112392F413
:106BE000F0E80F26FFEFE094F09400951095B09434
:106BF000C094D094A194BF0ACF0ADF0AEF0AFF0A1B
:106C00000F0B1F0B0E941A3607FC0E946B36CDB784
:106C1000DEB7ECE00C94A833689401C0E8948F923E
:106C20009F92CF93DF930E941A36DF91CF919F906E
:106C30008F90089588249924F401E401B0E49F938F
:106C4000AA279A158B049C04ED05FE05CF05D007F5
:106C5000A10798F4AD2FDC2FCF2FFE2FE92D982C14
:106C6000892E982F872F762F652F542F432F322F61
:106C70002227B85031F7BF9127C01B2EBF91BB27E9
:106C8000220F331F441F551F661F771F881F991F30
:106C9000881C991CEE1FFF1FCC1FDD1FAA1FBB1FE6
:106CA0008A149B04EC05FD05CE05DF05A007B1079E
:106CB00048F08A189B08EC09FD09CE09DF09A00BF2
:106CC000B10B21601A94E1F62EF49401AF01BE01DC
:106CD000CD01000C08956095709580959095309544
:106CE0004095509521953F4F4F4F5F4F6F4F7F4FCE
:106CF0008F4F9F4F0895002E083090F0982F872FC8
:106D0000762F652F542F432F322F22270850F4CF90
:106D1000220F331F441F551F661F771F881F991F9F
:106D20000A95B2F7002D089597FD1094002E0830B3
:106D300098F00850232F342F452F562F672F782F88
:106D4000892F912DF4CF1594979587957795679511
:106D500057954795379527950A95AAF71124002D41
:106D600008952A0D3B1D4C1D5D1D6E1D7F1D801F4E
:106D7000911F08952A153B054C055D056E057F059D
:106D80008007910708950024A7FD00942A17300575
:106D90004005500560057005800590050895AA1B03
:106DA000BB1B51E107C0AA1FBB1FA617B70710F0F6
:106DB000A61BB70B881F991F5A95A9F78095909528
:106DC000BC01CD010895EE0FFF1F0590F491E02D59
:106DD00009940F931F93CF93DF938230910510F4A2
:106DE00082E090E0E0913507F091360730E020E056
:106DF000B0E0A0E0309799F42115310509F44AC0BC
:106E0000281B390B24303105D8F58A819B81611507
:106E1000710589F1FB0193838283FE0111C04081DA
:106E200051810281138148175907E0F0481759072B
:106E300099F4109761F012960C93129713961C9385
:106E40003296CF01DF91CF911F910F91089500935A
:106E5000350710933607F4CF2115310551F042174D
:106E6000530738F0A901DB019A01BD01DF01F801E8
:106E7000C1CFEF01F9CF9093360780933507CDCF7F
:106E8000FE01E20FF31F8193919322503109398360
:106E90002883D7CF2091330730913407232B41F437
:106EA0002091C6013091C7013093340720933307F6
:106EB0002091C4013091C5012115310541F42DB750
:106EC0003EB74091C8015091C901241B350BE09198
:106ED0003307F0913407E217F307A0F42E1B3F0BA2
:106EE0002817390778F0AC014E5F5F4F241735073C
:106EF00048F04E0F5F1F5093340740933307819340
:106F000091939FCFF0E0E0E09CCFCF93DF93009789
:106F1000E9F0FC01329713821282A0913507B091FB
:106F20003607ED0130E020E01097A1F42081318197
:106F3000820F931F209133073091340728173907A8
:106F400009F061C0F0933407E0933307DF91CF91EC
:106F50000895EA01CE17DF07E8F54A815B819E01BB
:106F600041155105B1F7E901FB83EA834991599134
:106F7000C40FD51FEC17FD0761F480819181029643
:106F8000840F951FE90199838883828193819B8374
:106F90008A83F0E0E0E012968D919C911397009720
:106FA000B9F52D913C911197CD010296820F931F57
:106FB00020913307309134072817390739F6309775
:106FC00051F51092360710923507B0933407A0930D
:106FD0003307BCCFD383C28340815181840F951F77
:106FE000C817D90761F44E5F5F4F88819981480FB8
:106FF000591F518340838A819B819383828321150A
:10700000310509F0B0CFF0933607E09335079ECFF6
:10701000FD01DC01C0CF13821282D7CFB0E0A0E027
:10702000E4E1F8E30C9488338C01009751F4CB0130
:107030000E94E9368C01C801CDB7DEB7E0E10C94BF
:10704000A433FC01E60FF71F9C0122503109E2171F
:10705000F30708F49DC0D901CD91DC911197C617B3
:10706000D70798F0C530D10530F3CE0104978617C5
:10707000970708F3C61BD70B2297C193D1936D9343
:107080007C93CF010E948537D6CF5B01AC1ABD0A35
:107090004C018C0E9D1EA0913507B0913607512CE6
:1070A000412CF12CE12C109731F580913307909110
:1070B00034078815990509F05CC04616570608F094
:1070C00058C08091C4019091C501009741F48DB7DB
:1070D0009EB74091C8015091C901841B950BE817D8
:1070E000F90708F055C0F0933407E0933307F9012E
:1070F00071836083A0CF8D919C91119712966C90B3
:10710000129713967C901397A815B90559F56C0141
:1071100042E0C40ED11CCA14DB0420F1AC014A19B0
:107120005B09DA011296159780F0628273825183AF
:107130004083D9016D937C93E114F10471F0D70180
:107140001396FC93EE93129776CF22968C0F9D1F89
:10715000F90191838083F301EFCFF0933607E09339
:10716000350769CF4816590608F42C017D01D30173
:107170009ACFCB010E94E9367C01009749F0AE011D
:10718000B8010E94CB38C8010E948537870153CFD0
:1071900010E000E050CFFB01DC0102C001900D9235
:1071A00041505040D8F70895FB01DC018D910190CA
:1071B00080190110D9F3990B0895FB01DC010190AE
:1071C0000D920020E1F7089510E0C2E6D0E004C07F
:1071D000FE010E94E3362196C336D107C9F7F89421
:0271E000FFCFDF
:1071E20070E9D700C0320A0320E0B201903B7E0171
:1071F200D03F4401407D140170E9D700406B9A00F2
:1072020010936B00D0B13700903A1C0079003C001B
:1072120040787D0194F903001F1115111D1D111FE6
:107222001F1115111515111F1F111D1D1D1D1D1FCC
:107232001F1117111515111F1F1117111D1D111FD8
:107242001F1515111D1D1D1F1F111D111D1D111FA4
:1072520070E9D70070E09A00B0196D00D0B1370024
:10726200903A1C00F401000005009301BE01EA01FE
:10727200FE01120226023A026C02BA02E4020C0376
:1072820048035C03720388039D03A103A403A803BC
:10729200AC0340420F00485B890001A05D890001F8
:1072A20070E9D700000037078000000204000300E5
:1072B200011003020000030201000600040006059B
:1072C20000200605040000000000E50445047204E5
:1072D2003205A30481049504000000003607090763
:1072E200A507E606EA00F606E70600000000BB096D
:1072F2004504A507360431487A20003130487A0027
:107302003530487A0031303048003530304800316D
:107312006B487A0031306B48003130306B00417578
:10732200746F006E616E00696E66006F7666004370
:107332006F72722E504C4C205369353335312020F8
:107342000020467265712042464F2020434C4B324A
:107352002000467265712043575F42464F20434CDE
:107362004B310043575F42464F20204F66662F4FF6
:107372006E203F004F666600202020202020202023
:1073820020202020202020004F6E20002020424676
:107392004F204F66662F4F6E203F20200020202076
:1073A200205348494654204357202020200020489B
:1073B2007A2020202020004564697420467265717D
:1073C2002051554152545A0020487A0020456469A0
:1073D2007420535F4C4556454C203F2000202050DE
:1073E200494E204130203D2000302042616C6C200B
:1073F2003D204F46462056464F2000332042616CC6
:107402006C3D20302E38206D6B56200036204261B4
:107412006C6C3D2036206D6B5620202000392042B6
:10742200616C6C3D203530206D6B56202000392B6D
:10743200323064423D20353030206D6B56200039A9
:107442002B343064423D2035303030206D6B560095
:10745200392B363064423D2035303030306D6B563A
:1074620000550053534220004C5342004357202002
:10747200004C4F41440052454320005357522020B4
:1074820020202020503D305720202020200053571C
:10749200523D0020503D005720202000FFFFFFFFFB
:1074A200FFFFFFFF072B363000FFFFFFFFFFFFFF4D
:1074B200FF072B353500FFFFFFFFFFFFFFFF072B05
:1074C200353000FFFFFFFFFFFFFFFF072B343500C2
:1074D200FFFFFFFFFFFFFFFF072B343000FFFFFF1F
:1074E200FFFFFFFFFF072B333500FFFFFFFFFFFF0B
:1074F200FFFF072B333000FFFFFFFFFFFFFFFF07F8
:107502002B323500FFFFFFFFFFFFFFFF072B32305B
:1075120000FFFFFFFFFFFFFFFF072B313500FFFFDB
:10752200FFFFFFFFFFFF072B313000FFFFFFFFFFD1
:10753200FFFFFF072B352000FFFFFFFFFFFFFFFFCD
:107542000720202000FFFFFFFFFFFFFF0620202073
:107552002000FFFFFFFFFFFF05202020202000FF6B
:10756200FFFFFFFF0420202020202000FFFFFFFF5D
:10757200032020202020202000FFFFFF02202020C7
:10758200202020202000FFFF01202020202020207A
:10759200202000FFFF20202020202020202020006B
:1075A200FF2020202020202020202020004C0055D9
:0875B2005342004641003B007A
:00000001FF
